:020000040000FA
:06000000E7EF39F01200E9
:06000800BFEF1BF0120027
:06005A0004000E7400001A
:10006000290200000800000016740000FE010000D4
:100070000200000018740000FE03000002000000EF
:0C008000FC730000E30000001200000010
:10011000D9CFE6FFE1CFD9FF030EE126DF6ADF503A
:10012000F90F69E2DF50220DF3CF00F0F4CF01F0B8
:10013000000E0026010E0122010E00C0DBFF020EA0
:1001400001C0DBFF010EDBCFE9FFE828DBCFEAFFD0
:10015000EF6A010EDBCFE9FFE828DBCFEAFF210ED3
:10016000E926000EEA22EF90010EDBCFE9FFE82836
:10017000DBCFEAFF210EE926000EEA22EF82010E14
:10018000DBCFE9FFE828DBCFEAFF210EE926000EEE
:10019000EA22EF84010EDBCFE9FFE828DBCFEAFF9C
:1001A000210EE926000EEA22EF98010EDBCFE9FFCF
:1001B000E828DBCFEAFF210EE926000EEA22EF96BF
:1001C000010EDBCFE9FFE828DBCFEAFF0F0EE926BF
:1001D000000EEA22EF68010EDBCFE9FFE828DBCF53
:1001E000EAFF1F0EE926000EEA22580EEE6E020EFE
:1001F000EF6EDF2A94D70101EE6B040EEF6FF06B08
:10020000F16BF26BF36BE15EE7CFD9FF1200D9CF50
:10021000E6FFE1CFD9FF030EE126DF6ADF50F90FD9
:1002200001E386D0DF50220DF3CF00F0F4CF01F0D0
:10023000000E0026010E0122010E00C0DBFF020E9F
:1002400001C0DBFF010EDBCFE9FFE828DBCFEAFFCF
:10025000EF506CE1010EDBCFE9FFE828DBCFEAFFCE
:10026000010EEF6EDBCFE9FFE828DBCFEAFF0B0ED4
:10027000E926000EEA22E9CF00F0EACF01F0FD0EF8
:10028000DBCF02F0E828DBCF03F000C0E9FF01C0BC
:10029000EAFF02C0EEFF03C0EDFF010EDBCFE9FF76
:1002A000E828DBCFEAFF0D0EE926000EEA22EE6A0F
:1002B000EF6A010EDBCFE9FFE828DBCFEAFFEE5261
:1002C000060EE926000EEA22EE6AEE6AEE6AEF6A90
:1002D000010EDBCFE9FFE828DBCFEAFF210EE9269C
:1002E000000EEA22EF80010EDBCFE9FFE828DBCF2A
:1002F000EAFF210EE926000EEA22EF96010EDBCF7F
:10030000E9FFE828DBCFEAFF0F0EE926000EEA221C
:10031000EF68010EDBCFE9FFE828DBCFEAFF210E13
:10032000E926000EEA22EF82DF5003D0DF2A76D7DB
:10033000FE0EF36E040EE15EE7CFD9FF1200D9CFB7
:10034000E6FFE1CFD9FFFE0EDB50220DF3CFE9FF30
:10035000F4CFEAFF000EE926010EEA22EF50040A6C
:1003600001E102D0000E01D0010EF36EE552E7CF9D
:10037000D9FF1200D9CFE6FFE1CFD9FF020EE12667
:10038000FE0EDB50220DF3CF00F0F4CF01F0000E93
:100390000026010E012200C0DFFF010E01C0DBFFBD
:1003A000000EDBCFE9FFE828DBCFEAFFEF50040ABD
:1003B0000FE0000EDBCF00F0E828DBCF01F000C03B
:1003C000E6FF01C0E6FF64EC0DF0E550E55087D094
:1003D000FE0EDB50E66EC9EC04F0E550E66AE66A14
:1003E000E668110EE66E000EDBCFE9FFE828DBCFF2
:1003F000EAFF180EE926000EEA22EECF00F0EECF5B
:1004000001F0EECF02F0EECF03F000C0E6FF01C036
:10041000E6FF02C0E6FF03C0E6FFDBCFE9FFE82806
:10042000DBCFEAFF140EE926000EEA22EECF04F03D
:10043000EECF05F0EECF06F0EECF07F004C0E6FFFA
:1004400005C0E6FF06C0E6FF07C0E6FFDBCFE9FF19
:10045000E828DBCFEAFF0D0EE926000EEA22EECFF8
:1004600008F0EECF09F008C0E6FF09C0E6FFDBCFD9
:10047000E9FFE828DBCFEAFF0B0EE926000EEA22AF
:10048000EECF0AF0EECF0BF00AC0E6FF0BC0E6FF9E
:10049000DBCFE9FFE828DBCFEAFFEE52E9CF0CF033
:1004A000EACF0DF00CC0E6FF0DC0E6FFFAEC07F056
:1004B000120EE15E000EDBCFE9FFE828DBCFEAFF9A
:1004C000140EE926000EEA22EE2AEE22EE22EF2298
:1004D000DBCFE9FFE828DBCFEAFF050EEF6E030E66
:1004E000E15EE7CFD9FF1200D9CFE6FFE1CFD9FF18
:1004F000020EE126FE0EDB50220DF3CF00F0F4CF0A
:1005000001F0000E0026010E012200C0DFFF010EE7
:1005100001C0DBFF000EDBCFE9FFE828DBCFEAFFFD
:100520000F0EE926000EEA22EF50FF0A01E10ED07D
:10053000000EDBCFE9FFE828DBCFEAFF210EE9263A
:10054000000EEA22EFB2010EE86602D0F36A14D17F
:10055000000EDBCFE9FFE828DBCFEAFF100EE9262B
:10056000000EEA22EECF00F0EECF01F000C0E6FF71
:1005700001C0E6FFDBCFE9FFE828DBCFEAFF0F0E83
:10058000E926000EEA22EF50E66E100EE66E000E2F
:10059000DBCFE9FFE828DBCFEAFF180EE926000EE3
:1005A000EA22EECF02F0EECF03F0EECF04F0EECF72
:1005B00005F002C0E6FF03C0E6FF04C0E6FF05C089
:1005C000E6FFDBCFE9FFE828DBCFEAFF140EE926E0
:1005D000000EEA22EECF06F0EECF07F0EECF08F0E5
:1005E000EECF09F006C0E6FF07C0E6FF08C0E6FF51
:1005F00009C0E6FFDBCFE9FFE828DBCFEAFF0D0EFD
:10060000E926000EEA22EECF0AF0EECF0BF00AC088
:10061000E6FF0BC0E6FFDBCFE9FFE828DBCFEAFF10
:100620000B0EE926000EEA22EECF0CF0EECF0DF015
:100630000CC0E6FF0DC0E6FFDBCFE9FFE828DBCF0B
:10064000EAFFEE52E9CF0EF0EACF0FF00EC0E6FF60
:100650000FC0E6FFFAEC07F0120EE15E000EDBCFF2
:10066000E9FFE828DBCFEAFF140EE926000EEA22B4
:10067000EECFF6F1EECFF7F1EECFF8F1EECFF9F1E4
:10068000DBCFE9FFE828DBCFEAFF100EE926000EFA
:10069000EA22EECFF4F1EECFF5F1DBCFE9FFE82867
:1006A000DBCFEAFF140EE926000EEA22E9CF00F0C4
:1006B000EACF01F0DBCFE9FFE828DBCFEAFF100E3D
:1006C000E926000EEA22EECF02F0EECF03F000C0E2
:1006D000E9FF01C0EAFF0250EE260350EE22000EB1
:1006E000EE22EE22DBCFE9FFE828DBCFEAFF140E93
:1006F000E926000EEA22EECFF6F1EECFF7F1EECFCB
:10070000F8F1EECFF9F1DBCFE9FFE828DBCFEAFF24
:10071000210EE926000EEA22EF92DBCFE9FFE8285E
:10072000DBCFEAFF210EE926000EEA22EF98DBCFAD
:10073000E9FFE828DBCFEAFF0F0EE926000EEA22E8
:10074000EF50E66EAEEC2AF0E550000EDBCFE9FF8D
:10075000E828DBCFEAFF0F0EE926000EEA22EF6859
:10076000DBCFE9FFE828DBCFEAFF210EE926000E08
:10077000EA22EF82010EF36E030EE15EE7CFD9FFAE
:100780001200D9CFE6FFE1CFD9FFFE0EDB50220DDC
:10079000F3CFE9FFF4CFEAFF000EE926010EEA22CB
:1007A0000F0EE926000EEA22EF50FF0A04E160EC8A
:1007B00029F0F35011D0FE0EDB50220DF3CFE9FFEC
:1007C000F4CFEAFF000EE926010EEA22210EE92607
:1007D000000EEA22EFB2010EF36EE552E7CFD9FF29
:1007E0001200D9CFE6FFE1CFD9FF040EE126FE0EBD
:1007F000DB50220DF3CF00F0F4CF01F0000E002605
:10080000010E0122020E00C0DBFF030E01C0DBFF60
:10081000020EDBCFE9FFE828DBCFEAFF0F0EE92667
:10082000000EEA22EF50FF0A3AE1020EDBCFE9FFA9
:10083000E828DBCFEAFF0F0EE926000EEA22EF6A76
:10084000020EDBCFE9FFE828DBCFEAFF0F0EE92637
:10085000000EEA22EF50E66E10EC2BF0E550020E8F
:10086000DBCFE9FFE828DBCFEAFF100EE926000E18
:10087000EA22EE6AEF6A280EE66EE66A020EDBCF27
:10088000E9FFE828DBCFEAFF0F0EE926000EEA2297
:10089000EF50E66EFEEC2AF0E550E550E550020E12
:1008A000DBCFE9FFE828DBCFEAFF100EE926000ED8
:1008B000EA22EECF00F0EECF01F000C0DFFF010E24
:1008C00001C0DBFF000EDBCF00F0E828DBCF01F03A
:1008D000C40E005C000E015802E3F36A55D0020E0C
:1008E000DBCFE9FFE828DBCFEAFF210EE926000E87
:1008F000EA22EF88FD0EDB50E66E4BEC2AF0E55065
:10090000020EDBCFE9FFE828DBCFEAFF100EE92675
:10091000000EEA22EECF00F0EECF01F000C0DFFFC4
:10092000010E01C0DBFFDE4ADF2ADD52020EDBCF03
:10093000E9FFE828DBCFEAFF100EE926000EEA22E5
:10094000E9CF00F0EACF01F0DBCF02F0E828DBCFFF
:1009500003F000C0E9FF01C0EAFF02C0EEFF03C0E0
:10096000EDFF000EDBCF00F0E828DBCF01F0C40E76
:10097000005C000E015806E3FE0EDB50E66E74ECE0
:1009800002F0E550010EF36E050EE15EE7CFD9FFF0
:100990001200D9CFE6FFE1CFD9FF020EE126FE0E0D
:1009A000DB50220DF3CF00F0F4CF01F0000E002653
:1009B000010E012200C0DFFF010E01C0DBFF000EAF
:1009C000DBCFE9FFE828DBCFEAFF210EE926000EA6
:1009D000EA22EFB6010EE86602D0F36A0FD024ECEB
:1009E0002AF0000EDBCFE9FFE828DBCFEAFF210E7B
:1009F000E926000EEA22EF96010EF36E030EE15E89
:100A0000E7CFD9FF1200D9CFE6FFE1CFD9FF020E21
:100A1000E126FE0EDB50220DF3CF00F0F4CF01F003
:100A2000000E0026010E012200C0DFFF010E01C0F2
:100A3000DBFF000EDBCFE9FFE828DBCFEAFF210E6A
:100A4000E926000EEA22EFB6010EE85044E0000E5F
:100A5000DBCFE9FFE828DBCFEAFF210EE926000E15
:100A6000EA22EFB4010EE85012E0280EE66EE66AC4
:100A7000BDEC2AF0E550E550000EDBCFE9FFE82899
:100A8000DBCFEAFF210EE926000EEA22EF94000EEA
:100A9000DBCFE9FFE828DBCFEAFF210EE926000ED5
:100AA000EA22EF88FA0EDBCF00F0E828DBCF01F076
:100AB00000C0E6FF01C0E6FFFC0EDBCF02F0E82835
:100AC000DBCF03F002C0E6FF03C0E6FFEEEC29F047
:100AD000040EE15E02D0F36AF46A030EE15EE7CF32
:100AE000D9FF1200D9CFE6FFE1CFD9FF020EE126F0
:100AF000FE0EDB50220DF3CF00F0F4CF01F0000E1C
:100B00000026010E012200C0DFFF010E01C0DBFF45
:100B1000000EDBCFE9FFE828DBCFEAFF210EE92654
:100B2000000EEA22EFB6010EE85062E0000EDBCFC5
:100B3000E9FFE828DBCFEAFF210EE926000EEA22D2
:100B4000EFB4010EE85012E0280EE66EE66ABDEC46
:100B50002AF0E550E550000EDBCFE9FFE828DBCFB7
:100B6000EAFF210EE926000EEA22EF94000EDBCF09
:100B7000E9FFE828DBCFEAFF120EE926000EEA22A1
:100B8000EE5010E1ED500EE124EC2AF0000EDBCF28
:100B9000E9FFE828DBCFEAFF210EE926000EEA2272
:100BA000EF9626D0000EDBCFE9FFE828DBCFEAFF87
:100BB000120EE926000EEA22EE06ED5AFC0EDBCFFD
:100BC00000F0E828DBCF01F000C0E6FF01C0E6FF3F
:100BD000B9EC29F0E550E5CF01F0E7CF00F0F35094
:100BE00000C0E9FF01C0EAFFEF6E010EF36E01D015
:100BF000F36A030EE15EE7CFD9FF1200D9CFE6FF1B
:100C0000E1CFD9FFFE0EDB50220DF3CFE9FFF4CF89
:100C1000EAFF000EE926010EEA22210EE926000E67
:100C2000EA22EFB6010EF36EE552E7CFD9FF1200CC
:100C30001200D9CFE6FFE1CFD9FF240EE126140E32
:100C4000E66EE66AD9CF00F0DACF01F000C0E6FF29
:100C500001C0E6FFEEEC29F0040EE15ED9CF00F012
:100C6000DACF01F000C0E6FF01C0E6FFB9EC0BF0FF
:100C7000E550E550FD0EDBCFE9FFE828DBCFEAFFCA
:100C8000060EE926000EEA22EECF00F0EECF01F0CC
:100C9000EECF02F0EECF03F0140E00C0DBFF150E16
:100CA00001C0DBFF160E02C0DBFF170E03C0DBFF27
:100CB000180E00C2DBFF190E01C2DBFF1A0E02C2C2
:100CC000DBFF1B0E03C2DBFF1C0EDB6A060EE76EAA
:100CD0001D0EE7CFDBFFFB0EDBCF00F0E828DBCFFC
:100CE00001F01E0E00C0DBFF1F0E01C0DBFF1E0E59
:100CF000DBCF02F0E828DBCF03F002C0E6FF03C041
:100D0000E6FF5EEC30F0F4CF01F0F3CF00F0E550F9
:100D1000E5501E0E00C0DBFF1F0E01C0DBFF0C0EF6
:100D2000E66EE66AD9CF02F0DACF03F0140E02269F
:100D300002C0E6FF03C0E6FF44EC31F0F4CF01F05F
:100D4000F3CF00F0040EE15E001E011E210E00C074
:100D5000DBFF220E01C0DBFF240EE66EE66ABDEC6F
:100D60002AF0E550E550210EDB50E66E4BEC2AF000
:100D7000E550220EDB50E66E4BEC2AF0E550140EE7
:100D8000E66EE66ABDEC2AF0E550E550FB0EDBCFDF
:100D900002F0E828DBCF03F002C0E6FF03C0E6FF65
:100DA000E3EC09F0F4CF01F0F3CF00F0E550E550AB
:100DB000210E00C0DBFF220E01C0DBFF210EDBCFC6
:100DC00000F0E828DBCF01F0100EDBCF02F0E828BE
:100DD000DBCF03F00050025C02E10150035803E056
:100DE00024EC2AF000D10C0EDB50E842E842E84245
:100DF000E8420F0B3F0BE846E846EC0F006E230E6F
:100E000000C0DBFFFB0EDBCF02F0E828DBCF03F0F6
:100E1000230EDB50025C006E0350016A0156140E73
:100E2000005E000E015AFB0E00C0DBFFFC0E01C08D
:100E3000DBFF0C0EDB50E842E842E842E8420F0BD1
:100E40003F0BE846E846006E016A140E0026000ECD
:100E5000012200C0E6FF01C0E6FFBDEC2AF0E5502C
:100E6000E550FD0EDBCF01F0E828DBCF02F001C03A
:100E7000E6FF02C0E6FFD9CF03F0DACF04F003C0EB
:100E8000E6FF04C0E6FF56EC0AF0040EE15EF3CF85
:100E900000F0200E00C0DBFFDB50020F01E280D02B
:100EA00024EC2AF0200EDB50FF0A01E09CD0D9CFC1
:100EB00000F0DACF01F0080E0026FB0EDBCF02F0C7
:100EC000E828DBCF03F000C0E9FF01C0EAFF0250D1
:100ED000EE260350EE22000EEE22EE220D0EDB5027
:100EE000E842010BE85004E10D0EDB50010BE85025
:100EF00009E0080ED926000EDE2ADE22DE22DD22DF
:100F00000A0ED95EE66AE66AE668040EE66EDBCF94
:100F100000F0050EDBCF01F0060EDBCF02F0070E6E
:100F2000DBCF03F000C0E6FF01C0E6FF02C0E6FF32
:100F300003C0E6FF080EDBCF04F0090EDBCF05F09F
:100F40000A0EDBCF06F00B0EDBCF07F004C0E6FF86
:100F500005C0E6FF06C0E6FF07C0E6FF000EDBCFD8
:100F600008F0E828DBCF09F008C0E6FF09C0E6FF7B
:100F7000020EDBCF0AF0E828DBCF0BF00AC0E6FF59
:100F80000BC0E6FFFD0EDBCF0CF0E828DBCF0DF049
:100F90000CC0E6FF0DC0E6FFFAEC07F0120E22D0FF
:100FA000FB0EDBCF00F0E828DBCF01F000C0E6FF4E
:100FB00001C0E6FFD9CF02F0DACF03F002C0E6FFAE
:100FC00003C0E6FFFD0EDBCF04F0E828DBCF05F021
:100FD00004C0E6FF05C0E6FF200EDB50E66E0BEC1A
:100FE0000EF0070EE15E010EF36E250EE15EE7CF17
:100FF000D9FF1200D9CFE6FFE1CFD9FF260EE126B7
:1010000060EC29F0F35001E1FBD7FB0EDBCF00F0E1
:10101000E828DBCF01F0020E00C0DBFF030E01C0A9
:10102000DBFFF90EDBCF00F0E828DBCF01F0040E88
:1010300000C0DBFF050E01C0DBFFF50EDBCF00F0CB
:10104000F60EDBCF01F0F70EDBCF02F0F80EDBCFB0
:1010500003F0060E00C0DBFF070E01C0DBFF080E29
:1010600002C0DBFF090E03C0DBFFF10EDBCF00F097
:10107000F20EDBCF01F0F30EDBCF02F0F40EDBCF8C
:1010800003F00A0E00C0DBFF0B0E01C0DBFF0C0EED
:1010900002C0DBFF0D0E03C0DBFF0F0EDB9CDB9EEF
:1010A0000E0EDB90DB92DB94DB96F00EDBCF00F0D4
:1010B0000F0E00C0DBFF18EC2BF0F4CF01F0F3CFE4
:1010C00000F0100E00C0DBFF110E01C0DBFF100EA0
:1010D000DBCF00F0E828DBCF01F000502808000E3D
:1010E00001540BE2D9CFE9FFDACFEAFF100EE9266F
:1010F000D80EEE26FF0EED2205D0100ED926DE6AA0
:10110000DD6AD95E120ED926DE6ADD6AD95E140E5A
:10111000D926DE6ADD6AD95ED9CF00F0DACF01F0D8
:10112000020E002600C0E6FF01C0E6FFB9EC0BF09E
:10113000E550E550D9CFE9FFDACFEAFFED0EE92619
:10114000140EEE26000EED22F00EDB50E8A21FD0AA
:10115000D9CFE9FFDACFEAFFED0EE926040EEE263D
:10116000000EED22020EE76E160EE7CFDBFF040E37
:10117000E76E170EE7CFDBFF180EDB6AFA0EE76E9D
:10118000190EE7CFDBFF0E0EDB98DB8A03D00E0EC5
:10119000DB88DB9ADB8CDB9E1A0E00C2DBFF1B0EAA
:1011A00001C2DBFF1C0E02C2DBFF1D0E03C2DBFF10
:1011B000FD0EDBCFE9FFE828DBCFEAFF060EE926CC
:1011C000000EEA22EECF00F0EECF01F0EECF02F0FB
:1011D000EECF03F01E0E00C0DBFF1F0E01C0DBFFD1
:1011E000200E02C0DBFF210E03C0DBFF220EDB6AF4
:1011F000060EE76E230EE7CFDBFFED0EDBCF00F030
:10120000E828DBCF01F0240E00C0DBFF250E01C073
:10121000DBFF240EDBCF02F0E828DBCF03F002C0B7
:10122000E6FF03C0E6FF5EEC30F0F4CF01F0F3CF51
:1012300000F0E550E550240E00C0DBFF250E01C094
:10124000DBFF0C0EE66EE66AD9CF02F0DACF03F0D0
:101250001A0E022602C0E6FF03C0E6FF44EC31F09E
:10126000F4CF01F0F3CF00F0040EE15E001E011E8A
:10127000120E00C0DBFF130E01C0DBFF120EDBCF2E
:1012800000F0E828DBCF01F000C0DFFF010E01C055
:10129000DBFFEF0EDB50FF0A02E1EF0EDB6A140EFC
:1012A000E66EE66AEF0EDB50E66EFEEC2AF0E550E5
:1012B000E550E550ED0EDBCF00F0E828DBCF01F084
:1012C00000C0E6FF01C0E6FF060EE66EFD0EDBCFB6
:1012D00002F0E828DBCF03F002C0E6FF03C0E6FF20
:1012E00000EC27F0050EE15E140EE66EE66AD9CF3B
:1012F00000F0DACF01F0020E002600C0E6FF01C0C8
:10130000E6FF81EC2AF0040EE15EF00EDB50E8A26D
:1013100011D0040EE66EE66AD9CF00F0DACF01F004
:10132000160E002600C0E6FF01C0E6FF81EC2AF0A1
:10133000040EE15E140EE66EE66AEF0EDB50E66E1A
:10134000FEEC2AF0E550E550E550ED0EDBCF02F063
:10135000E828DBCF03F002C0E6FF03C0E6FFE3ECC2
:1013600009F0F4CF01F0F3CF00F0E550E55000C0F4
:10137000DFFF010E01C0DBFF240EE66EE66AEF0E12
:10138000DB50E66EFEEC2AF0E550E550E550010E2C
:10139000DB50E66E4BEC2AF0E550DF50E66E4BEC8E
:1013A0002AF0E550E66AE66AEF0EDB50E66EFEECE8
:1013B0002AF0E550E550E550A5EC2AF0270EE15E55
:1013C000E7CFD9FF1200D9CFE6FFE1CFD9FF040E56
:1013D000E126010EDF6EDE52DE6ADD6ADD52FD0EB1
:1013E000DBCF00F0DB06FE0EDBCF01F001E2DB0617
:1013F000005001E1015042E0B9EC29F0F3CF00F0D8
:10140000030E00C0DBFFDF5018E1030EDBCF02F05C
:10141000010EDB500224016E010E01C0DBFFDB5028
:10142000006E030EDB50005C1FE2020EDB2ADB5075
:10143000E8661AD0010EDB2A17D0030EDBCF02F0CC
:10144000020EDB500224016E020E01C0DBFFDB50F6
:10145000006E030EDB50005C07E2010EDB2ADB505E
:10146000E86602D0020EDB2ADF50E86602D0010EE9
:1014700001D0000E006E00C0DFFFB1D7020EDB50BE
:10148000E81C006E020E00C0DBFF010EDB50E81C02
:10149000006E010E00C0DBFFDBCFF3FFE828DBCFDF
:1014A000F4FF050EE15EE7CFD9FF1200D9CFE6FFCA
:1014B000E1CFD9FF040EE126FE0EE76E030EE7CF63
:1014C000DBFF020EDB6A020EDB50F90F01E3A0D056
:1014D000020EDB50220DF3CF00F0F4CF01F0000E2E
:1014E0000026010E012200C0DFFF010E01C0DBFF5C
:1014F000000EDBCFE9FFE828DBCFEAFFEF5001E188
:1015000084D0000EDBCFE9FFE828DBCFEAFF0B0E2B
:10151000E926000EEA22EECF00F0EECF01F0FD0E3C
:10152000DBCFE9FFE828DBCFEAFFEE52EE52EECF49
:1015300002F0EECF03F00050025C01E066D00150F3
:10154000035863E1000EDBCFE9FFE828DBCFEAFFB9
:10155000EF50010A06E1020EDBCF00F0030E00C0DF
:10156000DBFF000EDBCFE9FFE828DBCFEAFF0D0E43
:10157000E926000EEA22EECF00F0EECF01F0FD0EDC
:10158000DBCFE9FFE828DBCFEAFFEECF02F0EECFBA
:1015900003F00050025C02E10150035801E035D035
:1015A000000EDBCFE9FFE828DBCFEAFFEE52060EA4
:1015B000E926000EEA22EECF04F0EECF05F0EECFE2
:1015C00006F0EECF07F0FB0EDBCFE9FFE828DBCF1C
:1015D000EAFF060EE926000EEA22EECF08F0EECF73
:1015E00009F0EECF0AF0EECF0BF000010451085CD9
:1015F00008E10551095805E106510A5802E1075171
:101600000B5801E002D0020EA5D0020EDB2A5BD7F8
:10161000030EDB50220DF3CF00F0F4CF01F0000EEB
:101620000026010E012200C0DFFF010E01C0DBFF1A
:10163000030EDB50FE0A01E18FD0000EDBCFE9FF85
:10164000E828DBCFEAFFEF50010AD87401E184D02B
:101650000A0EE66EE66AFB0EDBCF00F0E828DBCF71
:1016600001F000C0E6FF01C0E6FF000EDBCFE9FF9E
:10167000E828DBCFEAFFEE52E9CF02F0EACF03F031
:1016800002C0E6FF03C0E6FF61EC37F0060EE15E44
:10169000000EDBCFE9FFE828DBCFEAFF0B0EE926DF
:1016A000000EEA22E9CF00F0EACF01F0FD0EDBCF19
:1016B000E9FFE828DBCFEAFFEE52EE52EECF02F070
:1016C000EECF03F000C0E9FF01C0EAFF02C0EEFF69
:1016D00003C0EDFF000EDBCFE9FFE828DBCFEAFF18
:1016E0000D0EE926000EEA22E9CF00F0EACF01F064
:1016F000FD0EDBCFE9FFE828DBCFEAFFEECF02F0FB
:10170000EECF03F000C0E9FF01C0EAFF02C0EEFF28
:1017100003C0EDFF000EDBCFE9FFE828DBCFEAFFD7
:10172000210EE926000EEA22EF96DBCFE9FFE8283A
:10173000DBCFEAFF0F0EE926000EEA22EF68DBCFCF
:10174000E9FFE828DBCFEAFF210EE926000EEA22B6
:10175000EF82030EDB5007D0030EDB50FE0A02E1DE
:10176000F36802D0FE0EF36E050EE15EE7CFD9FFFF
:101770001200D9CFE6FFE1CFD9FFFD0EDBCFE9FFA5
:10178000E828DBCFEAFFE9CF00F0EACF01F000C0A4
:10179000E6FF01C0E6FFFD0EDBCFE9FFE828DBCF67
:1017A000EAFFEECF04F0EECF05F004C0E6FF05C07F
:1017B000E6FF5EEC30F0F4CF03F0F3CF02F0E5503B
:1017C000E550E550E5CF01F0E7CF00F000C0E9FFBC
:1017D00001C0EAFF02C0EEFF03C0EDFFFD0EDBCF4C
:1017E000E9FFE828DBCFEAFFEE52EE52E9CF00F046
:1017F000EACF01F000C0E6FF01C0E6FFFD0EDBCF3F
:10180000E9FFE828DBCFEAFFEE52EE52EECF04F01C
:10181000EECF05F004C0E6FF05C0E6FF5EEC30F059
:10182000F4CF03F0F3CF02F0E550E550E550E5CFFB
:1018300001F0E7CF00F000C0E9FF01C0EAFF02C0FD
:10184000EEFF03C0EDFFFD0EDBCFE9FFE828DBCFA5
:10185000EAFF040EE926000EEA22E9CF00F0EACF03
:1018600001F000C0E6FF01C0E6FFFD0EDBCFE9FF9F
:10187000E828DBCFEAFF040EE926000EEA22EECFCD
:1018800006F0EECF07F0EECF08F0EECF09F006C07D
:10189000E6FF07C0E6FF08C0E6FF09C0E6FF89ECE7
:1018A00030F0EECF02F0EECF03F0EECF04F0EECF4B
:1018B00005F0040EE15EE550E5CF01F0E7CF00F062
:1018C00000C0E9FF01C0EAFF02C0EEFF03C0EEFF67
:1018D00004C0EEFF05C0EFFFFD0EDBCFE9FFE828F7
:1018E000DBCFEAFF080EE926000EEA22E9CF00F07E
:1018F000EACF01F000C0E6FF01C0E6FFFD0EDBCF3E
:10190000E9FFE828DBCFEAFF080EE926000EEA220D
:10191000EECF06F0EECF07F0EECF08F0EECF09F0F5
:1019200006C0E6FF07C0E6FF08C0E6FF09C0E6FF05
:1019300089EC30F0EECF02F0EECF03F0EECF04F002
:10194000EECF05F0040EE15EE550E5CF01F0E7CF04
:1019500000F000C0E9FF01C0EAFF02C0EEFF03C0D3
:10196000EEFF04C0EEFF05C0EFFFFD0EDBCFE9FF89
:10197000E828DBCFEAFF0E0EE926000EEA22E9CFC7
:1019800000F0EACF01F000C0E6FF01C0E6FFFD0E67
:10199000DBCFE9FFE828DBCFEAFF0E0EE926000ED9
:1019A000EA22EECF04F0EECF05F004C0E6FF05C05A
:1019B000E6FF5EEC30F0F4CF03F0F3CF02F0E55039
:1019C000E550E550E5CF01F0E7CF00F000C0E9FFBA
:1019D00001C0EAFF02C0EEFF03C0EDFFFD0EDBCF4A
:1019E000E9FFE828DBCFEAFF100EE926000EEA2225
:1019F000E9CF00F0EACF01F000C0E6FF01C0E6FF4A
:101A0000FD0EDBCFE9FFE828DBCFEAFF100EE92669
:101A1000000EEA22EECF04F0EECF05F004C0E6FFA0
:101A200005C0E6FF5EEC30F0F4CF03F0F3CF02F038
:101A3000E550E550E550E5CF01F0E7CF00F000C0FC
:101A4000E9FF01C0EAFF02C0EEFF03C0EDFFFD0E9B
:101A5000DBCFE9FFE828DBCFEAFF120EE926000E14
:101A6000EA22E9CF00F0EACF01F000C0E6FF01C0B2
:101A7000E6FFFD0EDBCFE9FFE828DBCFEAFF120E21
:101A8000E926000EEA22EECF04F0EECF05F004C006
:101A9000E6FF05C0E6FF5EEC30F0F4CF03F0F3CFD5
:101AA00002F0E550E550E550E5CF01F0E7CF00F05A
:101AB00000C0E9FF01C0EAFF02C0EEFF03C0EDFF76
:101AC000E552E7CFD9FF1200D9CFE6FFE1CFD9FF2A
:101AD000FD0EDBCFE9FFE828DBCFEAFF0F0EE9269A
:101AE000000EEA22EF50FF0A25E0FD0EDBCFE9FFF2
:101AF000E828DBCFEAFF0F0EE926000EEA22EF50BE
:101B0000E66EAEEC2AF0E550FD0EDBCFE9FFE828EB
:101B1000DBCFEAFF0F0EE926000EEA22EF68FD0E8A
:101B2000DBCFE9FFE828DBCFEAFF210EE926000E34
:101B3000EA22EF82FD0EDBCFE9FFE828DBCFEAFFE8
:101B4000EE52060EE926000EEA22EE6AEE6AEE6A10
:101B5000EF6AFD0EDBCFE9FFE828DBCFEAFF0D0ED1
:101B6000E926000EEA22EE6AEF6AFD0EDBCFE9FFFE
:101B7000E828DBCFEAFF210EE926000EEA22EFB6C5
:101B8000010EE85002E024EC2AF0FD0EDBCFE9FF65
:101B9000E828DBCFEAFF210EE926000EEA22EF96C5
:101BA000FD0EDBCFE9FFE828DBCFEAFF1F0EE926B9
:101BB000000EEA22580EEE6E020EEF6EFD0EDBCF27
:101BC000E9FFE828DBCFEAFF210EE926000EEA2232
:101BD000EF98FD0EDBCFE9FFE828DBCFEAFF210E0F
:101BE000E926000EEA22EF50010BE85009E0FD0E55
:101BF000DBCFE9FFE828DBCFEAFF010EEF6E07D06D
:101C0000FD0EDBCFE9FFE828DBCFEAFFEF6AE55204
:101C1000E7CFD9FF1200D9CFE6FFE1CFD9FF130EEE
:101C2000E126120EDB6AFE0EDB50220DF3CF00F030
:101C3000F4CF01F0000E0026010E0122100E00C0AC
:101C4000DBFF110E01C0DBFF100EDBCFE9FFE82840
:101C5000DBCFEAFF180EE926000EEA22EECF00F0F5
:101C6000EECF01F0EECF02F0EECF03F0080E00C091
:101C7000DBFF090E01C0DBFF0A0E02C0DBFF0B0E0B
:101C800003C0DBFF100EDBCFE9FFE828DBCFEAFF64
:101C9000140EE926000EEA22EECF00F0EECF01F09E
:101CA000EECF02F0EECF03F00C0E00C0DBFF0D0E06
:101CB00001C0DBFF0E0E02C0DBFF0F0E03C0DBFF17
:101CC000FA0EDBCFE9FFE828DBCFEAFF040EE926B6
:101CD000000EEA22EECF00F0EECF01F0EECF02F0E0
:101CE000EECF03F000C0DEFF01C0DDFF020E02C038
:101CF000DBFF030E03C0DBFFD9CF00F0DACF01F02A
:101D0000F80EDBCF02F0E828DBCF03F000C0E9FFDC
:101D100001C0EAFF0250EE260350EE22000EEE2232
:101D2000EE22100EDBCFE9FFE828DBCFEAFF140E2E
:101D3000E926000EEA22EECF00F0EECF01F0EECF62
:101D400002F0EECF03F0040E00C0DBFF050E01C071
:101D5000DBFF060E02C0DBFF070E03C0DBFFFA0E3F
:101D6000DBCFE9FFE828DBCFEAFF080EE926000E0B
:101D7000EA22EECFFAF1EECFFBF1EECFFCF1EECF9F
:101D8000FDF1100EDBCFE9FFE828DBCFEAFF1C0EE8
:101D9000E926000EEA22EF6A100EDBCFE9FFE82801
:101DA000DBCFEAFF1D0EE926000EEA22E9CF00F0A4
:101DB000EACF01F000C0E6FF01C0E6FFC5EC39F054
:101DC000F4CF03F0F3CF02F0E550E5CF01F0E7CF19
:101DD00000F000C0E9FF01C0EAFF02C0EEFF03C04F
:101DE000EDFF100EDBCFE9FFE828DBCFEAFF1F0E87
:101DF000E926000EEA22580EEE6E020EEF6E100E6D
:101E0000DBCFE9FFE828DBCFEAFFEF50010A01E072
:101E100016D124EC2AF0100EDBCFE9FFE828DBCF47
:101E2000EAFF140EE926000EEA22E9CF00F0EACF1D
:101E300001F00101F02BF123F223F32300C0E9FFAD
:101E400001C0EAFFF0C1EEFFF1C1EEFFF2C1EEFF0B
:101E5000F3C1EFFF100EDBCFE9FFE828DBCFEAFF8D
:101E6000180EE926000EEA22E9CF00F0EACF01F0D1
:101E7000DE2ADE22DE22DF22DDCF05F0DDCF04F018
:101E8000DDCF03F0DFCF02F000C0E9FF01C0EAFFC1
:101E900002C0EEFF03C0EEFF04C0EEFF05C0EFFF7F
:101EA000100EDBCFE9FFE828DBCFEAFF140EE926AE
:101EB000000EEA22EECF00F0EECF01F0EECF02F0FE
:101EC000EECF03F0040E00C0DBFF050E01C0DBFF08
:101ED000060E02C0DBFF070E03C0DBFF100EDBCFD8
:101EE000E9FFE828DBCFEAFF140EE926000EEA221C
:101EF000EE2AEE22EE22EF22FA0EDBCFE9FFE828EF
:101F0000DBCFEAFF0D0EE926000EEA22EFB2010E4A
:101F1000E8504EE00A0EE66EE66AFC0EDBCF00F0FB
:101F2000E828DBCF01F000C0E6FF01C0E6FF100E9D
:101F3000DBCFE9FFE828DBCFEAFFEE52E9CF02F082
:101F4000EACF03F002C0E6FF03C0E6FF61EC37F022
:101F5000060EE15E100EDBCFE9FFE828DBCFEAFFDB
:101F60000D0EE926000EEA22E9CF00F0EACF01F0DB
:101F7000FA0EDBCFE9FFE828DBCFEAFFEECF02F075
:101F8000EECF03F000C0E9FF01C0EAFF02C0EEFFA0
:101F900003C0EDFF120EE76EE7CFDBFF100EDBCFC5
:101FA000E9FFE828DBCFEAFF020EEF6EFAEF13F04D
:101FB000040EE76E120EE7CFDBFFDECF00F0DDCFC1
:101FC00001F0020EDBCF02F0030EDBCF03F0040EB4
:101FD00000C0DBFF050E01C0DBFF060E02C0DBFF09
:101FE000070E03C0DBFFFA0EDBCFE9FFE828DBCFEB
:101FF000EAFF040EE926000EEA22EECF00F0EECF53
:1020000001F0EECF02F0EECF03F000C0DEFF01C022
:10201000DDFF020E02C0DBFF030E03C0DBFF100E6C
:10202000DBCFE9FFE828DBCFEAFFEE52060EE92618
:10203000000EEA22EE6AEE6AEE6AEF6ADBD3FA0E6F
:10204000DBCFE9FFE828DBCFEAFF0D0EE926000E23
:10205000EA22EFB4010EE85012E024EC2AF0100E50
:10206000DBCF00F0E828DBCF01F000C0E6FF01C0C5
:10207000E6FF64EC0DF0E550E55056EF14F0040E69
:10208000DBCF00F0050EDBCF01F0060EDBCF02F058
:10209000070EDBCF03F0FA0EDBCFE9FFE828DBCF3A
:1020A000EAFF080EE926000EEA22EECF04F0EECF9A
:1020B00005F0EECF06F0EECF07F00050045C01E033
:1020C00097D30150055801E093D30250065801E020
:1020D0008FD30350075801E08BD3100EDBCFE9FFFD
:1020E000E828DBCFEAFFEF50020A01E078D0FA0ED1
:1020F000DBCFE9FFE828DBCFEAFF0D0EE926000E73
:10210000EA22EFB8010EE85001E172D3100EDBCFE6
:10211000E9FFE828DBCFEAFF180EE926000EEA22E5
:10212000E9CF00F0EACF01F0DECF02F0DDCF03F01F
:10213000020EDBCF04F0030EDBCF05F000C0E9FF99
:1021400001C0EAFF02C0EEFF03C0EEFF04C0EEFFD5
:1021500005C0EFFF100EDBCFE9FFE828DBCFEAFF79
:102160001C0EE926000EEA22EF6A100EDBCFE9FF13
:10217000E828DBCFEAFF1D0EE926000EEA22E9CFB0
:1021800000F0EACF01F000C0E6FF01C0E6FFC5ECB9
:1021900039F0F4CF03F0F3CF02F0E550E5CF01F0D2
:1021A000E7CF00F000C0E9FF01C0EAFF02C0EEFF88
:1021B00003C0EDFF100EDBCFE9FFE828DBCFEAFF1D
:1021C000040EEF6EF80EDBCF00F0E828DBCF01F055
:1021D00000500008000E015401E30AD39ED0100EF7
:1021E000DBCFE9FFE828DBCFEAFFEF50030A01E08D
:1021F000C7D0FA0EDBCFE9FFE828DBCFEAFF0D0EF0
:10220000E926000EEA22EFB2010EE85001E1F0D219
:10221000100EDBCFE9FFE828DBCFEAFF180EE92636
:10222000000EEA22E9CF00F0EACF01F0DE2ADE223A
:10223000DE22DF22DDCF05F0DDCF04F0DDCF03F0BD
:10224000DFCF02F000C0E9FF01C0EAFF02C0EEFFED
:1022500003C0EEFF04C0EEFF05C0EFFFFA0EDBCFB8
:10226000E9FFE828DBCFEAFF0D0EE926000EEA229F
:10227000EFB8010EE8500EE0100EE76E120EE7CF39
:10228000DBFF100EDBCFE9FFE828DBCFEAFF040E0F
:10229000EF6E37D0120EE76EE7CFDBFF100EDBCF0D
:1022A000E9FFE828DBCFEAFF020EEF6E100EDBCF6E
:1022B000E9FFE828DBCFEAFF140EE926000EEA2248
:1022C000E9CF00F0EACF01F0040ED926000EDE2A95
:1022D000DE22DE22DF22DDCF05F0DDCF04F0DDCF10
:1022E00003F0DFCF02F0040ED95E00C0E9FF01C0A9
:1022F000EAFF02C0EEFF03C0EEFF04C0EEFF05C020
:10230000EFFFF80EDBCF00F0E828DBCF01F0005044
:102310000008000E015401E36BD2100EDBCFE9FF81
:10232000E828DBCFEAFF210EE926000EEA22EF863D
:10233000100EDBCFE9FFE828DBCFEAFF120EE9261B
:10234000000EEA22E9CF00F0EACF01F0F80EDBCF71
:1023500002F0E828DBCF03F000C0E9FF01C0EAFF8C
:1023600002C0EEFF03C0EDFF100EDBCFE9FFE8284F
:10237000DBCFEAFF210EE926000EEA22EF843AD2F3
:10238000FA0EDBCFE9FFE828DBCFEAFF040EE926EF
:10239000000EEA22EECF00F0EECF01F0EECF02F019
:1023A000EECF03F0100EDBCFE9FFE828DBCFEAFF2A
:1023B000180EE926000EEA22EECF04F0EECF05F06B
:1023C000EECF06F0EECF07F00050045C08E10150BC
:1023D000055805E10250065802E10350075803E092
:1023E00024EC2AF063D2100EDBCFE9FFE828DBCF24
:1023F000EAFF180EE926000EEA22E9CF00F0EACF44
:1024000001F0DECF02F0DDCF03F0020EDBCF04F0EF
:10241000030EDBCF05F000C0E9FF01C0EAFF02C0F8
:10242000EEFF03C0EEFF04C0EEFF05C0EFFF100E8D
:10243000DBCFE9FFE828DBCFEAFFEF50040A01E039
:102440003ED1FA0EDBCFE9FFE828DBCFEAFF0D0E25
:10245000E926000EEA22EFB8010EE85032E0100E35
:10246000DBCFE9FFE828DBCFEAFF0F0EE926000EFD
:10247000EA22EF50FF0A25E0100EDBCFE9FFE82843
:10248000DBCFEAFF0F0EE926000EEA22EF50E66EE0
:10249000AEEC2AF0E550100EDBCFE9FFE828DBCFE9
:1024A000EAFF0F0EE926000EEA22EF68100EDBCFDE
:1024B000E9FFE828DBCFEAFF210EE926000EEA2239
:1024C000EF82FA0EDBCFE9FFE828DBCFEAFF0D0E43
:1024D000E926000EEA22EF50010BE8504FE0110E02
:1024E000E76E120EE7CFDBFF100EDBCFE9FFE82827
:1024F000DBCFEAFF140EE926000EEA22EECF00F051
:10250000EECF01F0EDCF02F0ED50000EEE2AEE22FC
:10251000EE22EF22040E00C0DBFF050E01C0DBFF40
:10252000060E02C0DBFF070E03C0DBFF100EDBCF81
:10253000E9FFE828DBCFEAFF180EE926000EEA22C1
:10254000EE2AEE22EE22EF22EDCF03F0EDCF02F0E5
:10255000EDCF01F0EFCF00F000C0DEFF01C0DDFFE6
:10256000020E02C0DBFF030E03C0DBFF100EDBCF49
:10257000E9FFE828DBCFEAFF0A0EEF6EF80EDBCFAB
:1025800000F0E828DBCF01F000500008000E0154F5
:1025900001E32ED1100EDBCFE9FFE828DBCFEAFF05
:1025A000210EE926000EEA22EFB6010EE86638D0C9
:1025B000100EDBCFE9FFE828DBCFEAFF210EE9268A
:1025C000000EEA22EF86100EDBCFE9FFE828DBCF12
:1025D000EAFF120EE926000EEA22E9CF00F0EACF68
:1025E00001F0F80EDBCF02F0E828DBCF03F000C0EB
:1025F000E9FF01C0EAFF02C0EEFF03C0EDFF100ECD
:10260000DBCFE9FFE828DBCFEAFF210EE926000E49
:10261000EA22EF84100EE76E120EE7CFDBFFEAD05E
:10262000120EDB6A100EDBCFE9FFE828DBCFEAFFF2
:10263000140EE926000EEA22E9CF00F0EACF01F0FD
:102640000C0EDBCF02F00D0EDBCF03F00E0EDBCF56
:1026500004F00F0EDBCF05F000C0E9FF01C0EAFF78
:1026600002C0EEFF03C0EEFF04C0EEFF05C0EFFFA7
:10267000100EDBCFE9FFE828DBCFEAFF180EE926D2
:10268000000EEA22E9CF00F0EACF01F0080EDBCF1E
:1026900002F0090EDBCF03F00A0EDBCF04F00B0EC5
:1026A000DBCF05F000C0E9FF01C0EAFF02C0EEFF8A
:1026B00003C0EEFF04C0EEFF05C0EFFF99D0100E7F
:1026C000DBCFE9FFE828DBCFEAFFEF500A0A12E18F
:1026D00024EC2AF0FA0EDBCFE9FFE828DBCFEAFF93
:1026E0000D0EE926000EEA22EFB8010EE85001E1D6
:1026F00081D06FD0100EDBCFE9FFE828DBCFEAFFF7
:10270000EF50050A4DE124EC2AF0FA0EDBCFE9FF89
:10271000E828DBCFEAFF0D0EE926000EEA22EF5093
:10272000010BE85067E0100EE76E120EE7CFDBFFFB
:10273000100EDBCFE9FFE828DBCFEAFF180EE92611
:10274000000EEA22EE2AEE22EE22EF22EDCF03F077
:10275000EDCF02F0EDCF01F0EFCF00F000C0DEFFD3
:1027600001C0DDFF020E02C0DBFF030E03C0DBFF72
:10277000FA0EDBCFE9FFE828DBCFEAFF0D0EE926F2
:10278000000EEA22EFB8010EE85001E022D0100E50
:10279000DBCFE9FFE828DBCFEAFF060EEF6E2AD099
:1027A000100EDBCFE9FFE828DBCFEAFFEF50060A87
:1027B00021E124EC2AF0FA0EDBCFE9FFE828DBCF99
:1027C000EAFF0D0EE926000EEA22EFB8010EE850EE
:1027D00011E0100EDBCF00F0E828DBCF01F000C0E5
:1027E000E6FF01C0E6FF64EC0DF0E550E55002D0D5
:1027F00024EC2AF0120EDB50000858E2E66AE66A82
:10280000E668120EDB50E66EDECF00F0DDCF01F0A1
:10281000020EDBCF02F0030EDBCF03F000C0E6FFB9
:1028200001C0E6FF02C0E6FF03C0E6FF040EDBCFF7
:1028300004F0050EDBCF05F0060EDBCF06F0070E29
:10284000DBCF07F004C0E6FF05C0E6FF06C0E6FFE9
:1028500007C0E6FFFA0EDBCFE9FFE828DBCFEAFF8F
:10286000EECF08F0EECF09F008C0E6FF09C0E6FFA2
:10287000FA0EDBCFE9FFE828DBCFEAFFEE52EE529B
:10288000EECF0AF0EECF0BF00AC0E6FF0BC0E6FF7A
:10289000FC0EDBCF0CF0E828DBCF0DF00CC0E6FF20
:1028A0000DC0E6FFFAEC07F0120EE15E140EE15ED9
:0628B000E7CFD9FF120082
:0A28B600D9CFE6FFE1CFD9FF010EF4
:1028C000E126DF6ADF50FB0F34E2DF500A0DF3CF61
:1028D000E9FFF4CFEAFF800EE926000EEA22E9CFF5
:1028E00000F0EACF01F000C0E6FF01C0E6FF500EA5
:1028F000E66EE66A07EC01F0E550E550E550E5CFFD
:1029000001F0E7CF00F0F35000C0E9FF01C0EAFF9B
:10291000EF6EDF500A0DF3CFE9FFF4CFEAFF800E30
:10292000E926000EEA22EE52EE52EE52EF6ADF2A5C
:10293000C9D7020EE15EE7CFD9FF1200D9CFE6FF7B
:10294000E1CFD9FF010EE126DF6ADF50FB0F07E27E
:10295000DF50E66EB4EC14F0E550DF2AF6D7020E35
:10296000E15EE7CFD9FF1200D9CFE6FFE1CFD9FF73
:10297000650EE126FE0EDB500A0DF3CF00F0F4CF1A
:1029800001F0800E0026000E0122610E00C0DBFF68
:10299000620E01C0DBFF010EE76E540EE7CFDBFFD6
:1029A000540EDB5001E117D3540EDB6A610EDBCF0E
:1029B000E9FFE828DBCFEAFFEF50E66E9FEC01F07D
:1029C000E550F3500BE1610EDBCFE9FFE828DBCFE8
:1029D000EAFFEE52EE52EE52EF6AFDD2610EDBCF0D
:1029E000E9FFE828DBCFEAFFEE52EE52EE52EF505D
:1029F000090A01E1BDD2080A01E184D20A0A01E113
:102A0000B2D1090A01E155D1020A01E0C9D7610E2C
:102A1000DBCFE9FFE828DBCFEAFFEF50E66EFEEC04
:102A200005F0E550F350BCE0010EE76E540EE7CF21
:102A3000DBFF520ED926DE6ADD6AD95E520EDBCF8D
:102A400000F0E828DBCF01F0500E005C000E0158CA
:102A500001E32FD000C0E6FF01C0E6FFD9CF04F0AC
:102A6000DACF05F0520EDBCF06F0DB2A530EDBCFB8
:102A700007F001E1DB2A06500424026E075005200E
:102A8000036E02C0E6FF03C0E6FF610EDBCFE9FF85
:102A9000E828DBCFEAFFEF50E66E72EC05F0E55078
:102AA000E550E550E550E5CF01F0E7CF00F0F350F9
:102AB000C5E1D9CF00F0DACF01F0520EDBCF02F042
:102AC000E828DBCF03F002500024E96E0350012018
:102AD000EA6EEF6A610EDBCFE9FFE828DBCFEAFFA1
:102AE000EF50E66EC9EC04F0E550610EDBCFE9FF74
:102AF000E828DBCFEAFFEE52EE52EE52020EEF6E06
:102B0000050EE76E5F0EE7CFDBFF610EDBCFE9FF5F
:102B1000E828DBCFEAFF090EE926000EEA22E9CF1A
:102B200001F0EACF02F001C0E6FF02C0E6FFD9CF14
:102B300003F0DACF04F05F0E032603C0E6FF04C003
:102B4000E6FFD9CF05F0DACF06F0550E052605C011
:102B5000E6FF06C0E6FFD9CF07F0DACF08F007C0DE
:102B6000E6FF08C0E6FF5FEC19F0080EE15EF3CF68
:102B700000F0510E00C0DBFFDB50E86611D75F0E9E
:102B8000DB5001081EE25F0EDB50E66ED9CF00F08D
:102B9000DACF01F0550E002600C0E6FF01C0E6FFC7
:102BA000CFEC1DF0E550E550E550610EDBCFE9FFBD
:102BB000E828DBCFEAFF090EE926000EEA22030E21
:102BC000EF6E610EDBCFE9FFE828DBCFEAFFEE52C4
:102BD000E9CF00F0EACF01F000C0E6FF01C0E6FF58
:102BE000550EDBCF04F0E828DBCF05F004C0E6FF8C
:102BF00005C0E6FF15EC32F0F4CF03F0F3CF02F09E
:102C0000E550E550E550E5CF01F0E7CF00F000C01A
:102C1000E9FF01C0EAFF02C0EEFF03C0EDFF610E55
:102C2000DBCFE9FFE828DBCFEAFFEE52EECF00F082
:102C3000EECF01F0FF0E005C0FE1FF0E01580CE13A
:102C4000610EDBCFE9FFE828DBCFEAFF080EE926BB
:102C5000000EEA22EF6A17D0610EDBCFE9FFE82809
:102C6000DBCFEAFFEE52EE5019E1ED5017E1610EB5
:102C7000DBCFE9FFE828DBCFEAFF080EE926000EEC
:102C8000EA22030EEF6E610EDBCFE9FFE828DBCF0F
:102C9000EAFFEE52EE52EE52020E9BD1610EDBCFF6
:102CA000E9FFE828DBCFEAFFEE52EE52EE520B0EC0
:102CB00090D1610EDBCFE9FFE828DBCFEAFFEF50D0
:102CC000E66EC1EC03F0E550F35001E169D6610E08
:102CD000DBCFE9FFE828DBCFEAFF080EE926000E8C
:102CE000EA22EF50020DF3CFE9FFF4CFEAFF290EFD
:102CF000E926020EEA22EECF00F0EECF01F0630EDD
:102D000000C0DBFF640E01C0DBFF630EDBCFF6FF0C
:102D1000DB2A640EDBCFF7FF01E1DB2A0A00F5CFE7
:102D200000F0600E00C0DBFFDB50E85010E0600EEA
:102D3000DB50E66E610EDBCFE9FFE828DBCFEAFF70
:102D4000EF50E66EF1EC03F0E550E550DED7610E92
:102D5000DBCFE9FFE828DBCFEAFFEF50E66E74EC4B
:102D600002F0E550FAD0610EDBCFE9FFE828DBCFB7
:102D7000EAFFEF50E66EC1EC03F0E550F35001E1DD
:102D80000FD6010EE76E540EE7CFDBFF600EDB6A55
:102D9000600EDB50E10F1AE2600EDBCFF6FFF76A40
:102DA000060EF626720EF7220800F550E66E610E4A
:102DB000DBCFE9FFE828DBCFEAFFEF50E66EF1EC6E
:102DC00003F0E550E550600EDB2AE2D7610EDBCF61
:102DD000E9FFE828DBCFEAFF090EE926000EEA2228
:102DE000EF50140DF3CFF6FFF4CFF7FF7A0EF6266F
:102DF000710EF722F6CF00F0F7CF01F0630E00C09E
:102E0000DBFF640E01C0DBFF630EDBCFF6FFDB2AC6
:102E1000640EDBCFF7FF01E1DB2A0A00F5CF00F0FB
:102E2000600E00C0DBFFDB50E85010E0600EDB50AE
:102E3000E66E610EDBCFE9FFE828DBCFEAFFEF505B
:102E4000E66EF1EC03F0E550E550DED7600EDB6A8C
:102E5000600EDB50FC0F1AE2600EDBCFF6FFF76A64
:102E6000260EF626720EF7220800F550E66E610E69
:102E7000DBCFE9FFE828DBCFEAFFEF50E66EF1ECAD
:102E800003F0E550E550600EDB2AE2D7610EDBCFA0
:102E9000E9FFE828DBCFEAFF090EE926000EEA2267
:102EA000EF50030A0DE1610EDBCFE9FFE828DBCF2D
:102EB000EAFF070EE926000EEA22010EEF6E0BD0A4
:102EC000610EDBCFE9FFE828DBCFEAFF070EE9263A
:102ED000000EEA22EF6A610EDBCFE9FFE828DBCFC4
:102EE000EAFF040EE926000EEA22030EEF6E610EE1
:102EF000DBCFE9FFE828DBCFEAFFEE52EE52EE52DD
:102F0000010E67D0610EDBCFE9FFE828DBCFEAFFD7
:102F1000EF50E66EFEEC05F0E550F3500BE0610E6D
:102F2000DBCFE9FFE828DBCFEAFFEF50E66EC9EC24
:102F300004F0E550610EDBCF00F0E828DBCF01F0B4
:102F400000C0E6FF01C0E6FFF0EC17F0E550E550E9
:102F5000F35001E125D5DEEC32F0610EDBCFE9FF65
:102F6000E828DBCFEAFFEE52EE52EE52090E31D0E6
:102F7000610EDBCFE9FFE828DBCFEAFFEF50E66E1A
:102F80009FEC01F0E550F35001E10AD5610EDBCF73
:102F9000E9FFE828DBCFEAFFEF50E66EC1EC03F073
:102FA000E550F35001E1FCD4610EDBCFE9FFE828E6
:102FB000DBCFEAFFEF50E66EBAEC01F0E550610EB0
:102FC000DBCFE9FFE828DBCFEAFFEE52EE52EE520C
:102FD0000A0EEF6EE5D4660EE15EE7CFD9FF120070
:102FE000D9CFE6FFE1CFD9FF020EE126FD0EDBCF00
:102FF000E9FFE828DBCFEAFFEE52EECF39F2EECF61
:103000003AF2FD0EDBCFE9FFE828DBCFEAFFEF5015
:10301000E66EC1EC03F0E550F35001E13FD1DF6A09
:10302000FD0EDBCFE9FFE828DBCFEAFF040EE9263F
:10303000000EEA22EF50080A1CE0E5EC32F0F3CF74
:1030400000F0010E00C0DBFF0201FF0E395D11E14F
:10305000FF0E3A590EE1FD0EDBCFE9FFE828DBCF8A
:10306000EAFFEF50E66E74EC02F0E550010EF36EED
:1030700021D1FD0EDBCFE9FFE828DBCFEAFF070E09
:10308000E926000EEA22EF5001E1F8D0FD0EDBCF79
:10309000E9FFE828DBCFEAFF040EE926000EEA226A
:1030A000EF50080A01E174D00E0A43E0030A16E06B
:1030B000060A01E0DFD0010EDB50250A0CE1FD0E0F
:1030C000DBCFE9FFE828DBCFEAFF040EE926000E9C
:1030D000EA22050ECDD0010EDF6ECDD0010EDB5001
:1030E000250A03E1010EDF6EB8D0FD0EDBCFE9FF4C
:1030F000E828DBCFEAFF080EE926000EEA22E9CF36
:1031000000F0EACF01F0010EDB50D00F0F0BE83AD0
:1031100000C0E9FF01C0EAFFEF6EFD0EDBCFE9FF63
:10312000E828DBCFEAFF040EE926000EEA22060EAD
:103130009FD0FD0EDBCFE9FFE828DBCFEAFF080ECA
:10314000E926000EEA22E9CF00F0EACF01F0010EF5
:10315000DB50D00F00C0E9FF01C0EAFFEF12FD0E07
:10316000DBCFE9FFE828DBCFEAFF040EE926000EFB
:10317000EA22080EEF6EFD0EDBCFE9FFE828DBCF79
:10318000EAFF050EE926000EEA22EE6AEF6A73D026
:10319000FD0EDBCFE9FFE828DBCFEAFF050EE926CD
:1031A000000EEA22E9CF00F0EACF01F000C0E6FF0E
:1031B00001C0E6FFD9CF04F0DACF05F0010E0426F6
:1031C00004C0E6FF05C0E6FFFD0EDBCFE9FFE828FF
:1031D000DBCFEAFF050EE926000EEA22EECF06F06D
:1031E000EECF07F006C0E6FF07C0E6FFFD0EDBCF1F
:1031F000E9FFE828DBCFEAFF080EE926000EEA2205
:10320000EF50E66E34EC1EF0F4CF03F0F3CF02F093
:10321000050EE15EE550E5CF01F0E7CF00F000C01C
:10322000E9FF01C0EAFF02C0EEFF03C0EDFF010E9F
:10323000DF6EFD0EDBCFE9FFE828DBCFEAFF050EEE
:10324000E926000EEA22EECF00F0EECF01F0FF0EED
:10325000005C11E1FF0E01580EE1FD0EDBCFE9FF2E
:10326000E828DBCFEAFF040EE926000EEA22030E6F
:10327000EF6E01D0FFD7DF5001E1C3D6010EDB5066
:10328000E66EFD0EDBCFE9FFE828DBCFEAFFEF506B
:10329000E66EF1EC03F0E550E550B3D6FD0EDBCF62
:1032A000E9FFE828DBCFEAFFEE5239C2EEFF3AC26F
:1032B000EDFFF36A030EE15EE7CFD9FF1200D9CF2D
:1032C000E6FFE1CFD9FF080EE126010EDB6A030E0F
:1032D000D926DE6ADD6AD95EDF6AE66EE66A2B0E03
:1032E000006E720E016E0001026B00C0E6FF01C0AD
:1032F000E6FF02C0E6FFFD0EDBCF03F0E828DBCFE0
:1033000004F003C0E6FF04C0E6FF41EC37F0070E0F
:10331000E15EF3500DE1D9CFE9FFDACFEAFFFD0E10
:10332000E926040EEE26000EED22020EDB6A31D0F5
:10333000040EE66EE66A2F0E006E720E016E00013C
:10334000026B00C0E6FF01C0E6FF02C0E6FFFD0E13
:10335000DBCF03F0E828DBCF04F003C0E6FF04C0B6
:10336000E6FF41EC37F0070EE15EF35010E1D9CFF4
:10337000E9FFDACFEAFFFD0EE926050EEE26000E84
:10338000ED22010EE76E020EE7CFDBFF02D0020E48
:10339000F0D1FD0EDBCFE9FFE828DBCFEAFFEF50ED
:1033A000200A06E1FD0EDB2AF4E1FE0EDB2AF1D74E
:1033B000FD0EDBCFE9FFE828DBCFEAFFEECF00F020
:1033C000050E00C0DBFFDB50200A01E10BD1050E2A
:1033D000DB50E85001E106D1050EDB500D0A01E19A
:1033E00001D1050EDB500A0A01E1FCD0DFCF00F06D
:1033F000F90EDBCFE9FFE828DBCFEAFFEF50005CF6
:1034000001E3F0D0010EDB50020A60E0030A39E06C
:10341000010A01E0E0D0FB0EDBCF02F0E828DBCFB1
:1034200003F0DF50020DF3CF04F0F4CF05F00450A9
:103430000224006E05500320016EFD0EDBCF06F066
:10344000E828DBCF07F000C0E9FF01C0EAFF06C0B3
:10345000EEFF07C0EDFFFD0EDBCFE9FFE828DBCF75
:10346000EAFFEECF00F0050E00C0DBFFDB502F0AB5
:10347000D87404E1050EDB505C0AD87401E1ABD0CE
:1034800040D0FB0EDBCF02F0E828DBCF03F0DF50AB
:10349000DF2A020DF3CF04F0F4CF05F0045002242C
:1034A000006E05500320016EFD0EDBCF06F0E8280C
:1034B000DBCF07F000C0E9FF01C0EAFF06C0EEFF66
:1034C00007C0EDFF020EE76E010E1DD0FD0EDBCF33
:1034D000E9FFE828DBCFEAFFEECF00F0050E00C0E1
:1034E000DBFFDB503F0AD87404E1050EDB50260AEF
:1034F000D8740CE0FD0EDBCFE9FFE828DBCFEAFF54
:10350000EF6A010EE76EE7CFDBFF65D0050EDB50FB
:103510002B0A09E1FD0EDBCFE9FFE828DBCFEAFF4C
:10352000200EEF6E58D0050EDB502E0A01E014D0AD
:10353000DF50010A01E010D0FD0EDB2ADBCF00F0E6
:10354000FE0E01E1DB2ADBCF01F0030E00C0DBFF42
:10355000040E01C0DBFF3FD0050EDB503D0A0CE13D
:10356000FD0EDBCFE9FFE828DBCFEAFFEF6A010EB3
:10357000E76EE7CFDBFF2FD0050EDB502F0AD874A4
:1035800004E1050EDB505C0AD87425E0FB0EDBCFAE
:1035900002F0E828DBCF03F0DF50FF0F020DF3CF7E
:1035A00004F0F4CF05F004500224006E055003200F
:1035B000016EFD0EDBCF06F0E828DBCF07F0010E31
:1035C0000626000E072200C0E9FF01C0EAFF06C080
:1035D000EEFF07C0EDFFFD0EDB2A01E0E9D6FE0E8F
:1035E000DB2AE6D6FD0EDBCFE9FFE828DBCFEAFFDA
:1035F000EF6AF70EDBCFE9FFE828DBCFEAFF070E23
:10360000EF6ED9CFE9FFDACFEAFF030EE926EE50DD
:1036100001E1ED5064E0030EDBCF02F0E828DBCFE0
:1036200003F002C0E6FF03C0E6FFE7EC37F0F4CF9B
:1036300001F0F3CF00F0E550E550030E00C0DBFFD2
:10364000040E01C0DBFF5E0E006E710E016E060EF1
:1036500000C0DBFF070E01C0DBFF050EDB6A050EB5
:10366000DB50F90F3CE2030EE66EE66A060EDBCF96
:1036700000F0E828DBCF01F00001026B00C0E6FF9C
:1036800001C0E6FF02C0E6FF030EDBCF03F0E8282F
:10369000DBCF04F003C0E6FF04C0E6FF41EC37F0E7
:1036A000070EE15EF3500EE1F70EDBCF00F0E828E5
:1036B000DBCF01F0050EDB5000C0E9FF01C0EAFFDF
:1036C000EF6E0DD0D9CFE9FFDACFEAFF060EE9267B
:1036D000040EEE26000EED22050EDB2AC0D7DF50C9
:1036E000E86639D0090EE66EE66A340E006E720E98
:1036F000016E0001026B00C0E6FF01C0E6FF02C0E0
:10370000E6FFFB0EDBCFE9FFE828DBCFEAFFEECFD9
:1037100003F0EECF04F003C0E6FF04C0E6FF8CEC3C
:1037200037F0070EE15EFB0EDBCFE9FFE828DBCFC9
:10373000EAFFEE50EDCFEAFFE96E090EE926000E32
:10374000EA22EF6AF70EDBCFE9FFE828DBCFEAFFDA
:10375000010EEF6EDF2AF90EDBCF00F0E828DBCF99
:1037600001F0DF5000C0E9FF01C0EAFFEF6E020E7A
:0E377000DB50F36E090EE15EE7CFD9FF1200C9
:02377E00DACFA0
:10378000E4FFE652E9CFE6FFEACFE6FF000EE96E7E
:10379000000EEA6E100EE80403E3EECFE6FFFBD75F
:1037A000CAEC39F06DEC28F0E5520F0EE96E000E10
:1037B000EA6E100EE80403E3E5CFEDFFFBD7E5CF9B
:1037C000EAFFE5CFE9FFE5CFDAFF1100D9CFE6FF49
:1037D000E1CFD9FFACB201D0FDD7FE0EDB50AD6E0C
:1037E000E552E7CFD9FF1200D9CFE6FFE1CFD9FFED
:1037F000010EE126FD0EDBCFE9FFDB2AFE0EDBCF5B
:10380000EAFF01E1DB2AEECF00F0000E00C0DBFF93
:10381000DB50E85006E0DF50E66EE6EC1BF0E550CA
:10382000E9D7020EE15EE7CFD9FF1200F86AEAECB1
:103830001EF0BBEC39F00FEC32F00BEC1FF081BA4C
:103840000FD0C00EE66E89EC35F0E550A90EE66E9D
:103850006C0EE66EFAEC35F0E550E5508DEC21F09B
:1038600036EC34F05BEC14F03FEC34F09EEC14F0EA
:1038700078EC1DF00001E451E35DF6E0010EE66E28
:10388000000E006E020E016E00C0E6FF01C0E6FFF2
:1038900065EC1CF0E550E550E550E4C0E3F00201B2
:1038A00018A1E2D7CE0EE66E89EC35F0E5500A0E8F
:1038B0000001E35D03E2E351300F02D0E351410F19
:1038C000E66E1FEC36F0E550CFD7D9CFE6FFE1CF5B
:1038D000D9FF080EE126FC0EDB5012E0C00EE66EAA
:1038E00089EC35F0E550B80EE66E6C0EE66EFAEC3B
:1038F00035F0E550E550C00EE66E89EC35F0E55048
:10390000D9CF00F0DACF01F000C0E6FF01C0E6FF3A
:10391000FD0EDBCFE9FFE828DBCFEAFFEECF02F0B8
:10392000036A02C0E6FF03C0E6FF9CEC33F0040E1E
:10393000E15EFC0EDB5011E0D9CF00F0DACF01F0F0
:1039400000C0E6FF01C0E6FFD6EC35F0E550E550DB
:103950002E0EE66E1FEC36F010D0D9CF00F0DACF85
:1039600001F000C0E6FF01C0E6FFF4EC1BF0E550FB
:10397000E5502E0EE66EE6EC1BF0E550D9CF00F0D8
:10398000DACF01F000C0E6FF01C0E6FFFD0EDBCF9D
:10399000E9FFE828DBCFEAFFEE52EECF02F0036A40
:1039A00002C0E6FF03C0E6FF9CEC33F0040EE15ECC
:1039B000FC0EDB5011E0D9CF00F0DACF01F000C0EF
:1039C000E6FF01C0E6FFD6EC35F0E550E5502E0EDF
:1039D000E66E1FEC36F010D0D9CF00F0DACF01F050
:1039E00000C0E6FF01C0E6FFF4EC1BF0E550E55037
:1039F0002E0EE66EE6EC1BF0E550D9CF00F0DACFE4
:103A000001F000C0E6FF01C0E6FFFD0EDBCFE9FFDD
:103A1000E828DBCFEAFFEE52EE52EECF02F0036A67
:103A200002C0E6FF03C0E6FF9CEC33F0040EE15E4B
:103A3000FC0EDB5011E0D9CF00F0DACF01F000C06E
:103A4000E6FF01C0E6FFD6EC35F0E550E5502E0E5E
:103A5000E66E1FEC36F010D0D9CF00F0DACF01F0CF
:103A600000C0E6FF01C0E6FFF4EC1BF0E550E550B6
:103A70002E0EE66EE6EC1BF0E550D9CF00F0DACF63
:103A800001F000C0E6FF01C0E6FFFD0EDBCFE9FF5D
:103A9000E828DBCFEAFFEE52EE52EE52EECF02F014
:103AA000036A02C0E6FF03C0E6FF9CEC33F0040E9D
:103AB000E15EFC0EDB500BE0D9CF00F0DACF01F075
:103AC00000C0E6FF01C0E6FFD6EC35F00AD0D9CF42
:103AD00000F0DACF01F000C0E6FF01C0E6FFF4EC31
:103AE0001BF0E550E550090EE15EE7CFD9FF12006B
:103AF000D9CFE6FFE1CFD9FF020EE126810EC26EDB
:103B0000640EDF6EDF50DF06E85001E0FBD7C284B1
:103B1000C2A401D0FDD7C3CFDFFF010EC4CFDBFFAE
:103B2000190EE66E020EE66E000EDBCF00F0E828FE
:103B3000DBCF01F000C0E6FF01C0E6FF9CEC33F0F4
:103B4000040EE15E840EC16E890EC26E640EDF6EDD
:103B5000DF50DF06E85001E0FBD7C284C2A401D0E9
:103B6000FDD7C3CFDFFF010EC4CFDBFF210EE66E12
:103B7000020EE66E000EDBCF00F0E828DBCF01F08E
:103B800000C0E6FF01C0E6FF9CEC33F0040EE15EEE
:103B90008E0EC16E030EE15EE7CFD9FF1200D9CFC2
:103BA000E6FFE1CFD9FF020EE126FD0EDBCFE9FFF4
:103BB000E828DBCFEAFFEE50EDCFEAFFE96EEF50E9
:103BC000D00F006E00C0DFFFDF50010A48E0010A9D
:103BD00001E024D0FD0EDBCFE9FFE828DBCFEAFFD0
:103BE000EE52EE52EE50EDCFEAFFE96EEF50D00FFD
:103BF000006E010E00C0DBFFDB50010A06E0010A87
:103C000001E005D00F01897602D00F0189740D0EF5
:103C1000E66EE66AC90E006E6C0E06D00A0EE66EFF
:103C2000E66AD60E006E6C0E016E0001026B00C0DB
:103C3000E6FF01C0E6FF02C0E6FFFD0EDBCFE9FFB5
:103C4000E828DBCFEAFFEECF03F0EECF04F003C0AD
:103C5000E6FF04C0E6FF8CEC37F0070EE15E030ED2
:103C6000E15EE7CFD9FF1200D9CFE6FFE1CFD9FF60
:103C7000FE0EDB50040A01E195D0070A4DE0010A6F
:103C80000BE0030A06E0010A01E09ED089A68CD071
:103C900093D089A489D090D0D9CFE9FFDACFEAFFB9
:103CA000FC0EE926EE5007E1ED5005E1FC0ED926A9
:103CB000DE6ADD6AD95EFA0EDBCF00F0E828DBCFE2
:103CC00001F0D9CFE9FFDACFEAFFFC0EE926EF5089
:103CD000EA6A190FE96E020EEA22EF5000C0E9FF0E
:103CE00001C0EAFFEF6ED9CFE9FFDACFEAFFFC0EA1
:103CF000E926EF50EA6A190FE96E020EEA22EF5048
:103D000001E162D0FC0EDBCF00F0DB2AFD0EDBCF41
:103D100001F041E1DB2A3FD0D9CFE9FFDACFEAFF5A
:103D2000FC0EE926EE5007E1ED5005E1FC0ED92628
:103D3000DE6ADD6AD95EFA0EDBCF00F0E828DBCF61
:103D400001F0D9CFE9FFDACFEAFFFC0EE926EF5008
:103D5000EA6A210FE96E020EEA22EF5000C0E9FF85
:103D600001C0EAFFEF6ED9CFE9FFDACFEAFFFC0E20
:103D7000E926EF50EA6A210FE96E020EEA22EF50BF
:103D800001E122D0FC0EDBCF00F0DB2AFD0EDBCF01
:103D900001F001E1DB2AFC0EDBCFF3FFE828DBCFEB
:103DA000F4FF14D081AA08D0FA0EDBCFE9FFE8288F
:103DB000DBCFEAFF310E07D0FA0EDBCFE9FFE828B0
:103DC000DBCFEAFF300EEF6EF368F468E552E7CF21
:103DD000D9FF12008E0EC16E030E926E809A8984F6
:103DE0008986F19E42EC35F0800EE66E89EC35F066
:103DF000E5509A0EE66E6C0EE66EFAEC35F0E55084
:103E0000E550200EAC6E900EAB6E0F0EAF6ED56A05
:103E1000F28EF28C120002010A0E006F016F050E85
:103E2000026F0F0E036F0A690B690C690D6B0A0EA6
:103E30000E6F0F6F050E106F0F0E116F046B040ED7
:103E4000056FA30E066F076B086B096B18911200C4
:103E5000D9CFE6FFE1CFD9FF010EE126FD0EDBCF82
:103E6000F6FFDB2AFE0EDBCFF7FF01E1DB2A0A00BB
:103E7000F5CF00F0000E00C0DBFFDB50E85006E09D
:103E8000DF50E66EE6EC1BF0E550E8D7020EE15E8F
:103E9000E7CFD9FF1200D9CFE6FFE1CFD9FF020E5D
:103EA000E126010EDB6A9EBA01D0FDD7AECFDFFF5F
:103EB000DF500D0AD87403E1DF500A0AD87401E01C
:103EC0001FD0010EDB2AFD0EDBCF00F0DB2AFE0E39
:103ED000DBCF01F001E1DB2ADF5000C0E9FF01C0C8
:103EE000EAFFEF6EFD0EDBCFE9FFE828DBCFEAFF4C
:103EF000EF6AFC0EDBCFE9FFDB06E950E866D3D7BB
:103F0000010EDB50F36E030EE15EE7CFD9FF120026
:103F1000D9CFE6FFE1CFD9FF040EE126FD0EDBCFBE
:103F200000F0E828DBCF01F0010E00C0DBFF020E3D
:103F300001C0DBFF030EDB6AFD0EDBCFE9FFE828E3
:103F4000DBCFEAFFEECF00F0000E00C0DBFFDB505E
:103F5000E85062E0DF502E0A50E1FD0EDBCFE9FFB2
:103F6000DB2AFE0EDBCFEAFF01E1DB2AEF6AFB0E64
:103F7000DBCFE9FFE828DBCFEAFFE9CF02F0EACFA9
:103F800003F0030EDBCFE9FFDB2AE950016A0224CC
:103F9000006E0350012200C0E6FF01C0E6FF02C030
:103FA000E6FF03C0E6FF010EDBCF04F0E828DBCF1D
:103FB00005F004C0E6FF05C0E6FF27EC33F0E5504E
:103FC000E550E550E5CF03F0E5CF02F0E5CF01F095
:103FD000E7CF00F0F35000C0E9FF01C0EAFFEF6E49
:103FE000FD0EDBCF00F0E828DBCF01F0010E00C0B2
:103FF000DBFF020E01C0DBFF09D0DF50D00F01E272
:1040000003D0DF50390802E2F36A45D0FD0EDB2A07
:1040100093E1FE0EDB2A90D7FB0EDBCFE9FFE82809
:10402000DBCFEAFFE9CF02F0EACF03F0030EDB506B
:10403000016A0224006E0350012200C0E6FF01C0A5
:10404000E6FF02C0E6FF03C0E6FF010EDBCF04F08F
:10405000E828DBCF05F004C0E6FF05C0E6FF27EC4B
:1040600033F0E550E550E550E5CF03F0E5CF02F041
:10407000E5CF01F0E7CF00F0F35000C0E9FF01C049
:10408000EAFFEF6E030EDB50030A01E102D0000EDF
:1040900001D0010EF36E050EE15EE7CFD9FF1200ED
:1040A000D9CFE6FFE1CFD9FF010EE1269EBA01D0BC
:1040B000FDD7AECFDFFFDF50CF0F01E206D0DF50DC
:1040C000C70F01E302D0DF5001D0390EF36E020EAC
:1040D000E15EE7CFD9FF1200D9CFE6FFE1CFD9FFEC
:1040E0001A0EE1260D0EE66EE6EC1BF0E5500A0E08
:1040F000E66EE6EC1BF0E550FE0EDB50D00FFF0F36
:10410000020DF3CFE9FFF4CFEAFFE50EE926000E3A
:10411000EA22EECF00F0EECF01F000C0E6FF01C0D2
:10412000E6FF28EC1FF0E550E550FE0EDB50380AA4
:1041300001E1EED00F0A01E1EBD0010A01E1E6D086
:10414000030A01E1E0D0010A60E0070A5AE0010A2F
:1041500054E0030A01E0DCD0D9CF00F0DACF01F05F
:1041600000C0E6FF01C0E6FF12C2E6FF13C2E6FF91
:104170009CEC33F0040EE15ED9CF00F0DACF01F011
:1041800000C0E6FF01C0E6FFF4EC1BF0E550E5508F
:10419000290EE66EE6EC1BF0E5503A0EE66EE6EC14
:1041A0001BF0E550200EE66EE6EC1BF0E550140E19
:1041B000E66ED9CF00F0DACF01F000C0E6FF01C013
:1041C000E6FF4BEC1FF0E550E550E550F3506DE095
:1041D000D9CF00F0DACF01F000C0E6FF01C0E6FF62
:1041E00027EC33F0F4CF13F2F3CF12F2E550E550A1
:1041F00013C208F212C209F28BD0000E006E020E3A
:1042000007D00E0E006E020E03D00A0E006E020ED4
:10421000016E180E00C0DBFF190E01C0DBFFE66A5D
:10422000180EDBCF00F0E828DBCF01F000C0E6FF7E
:1042300001C0E6FF65EC1CF0E550E550E550290EA5
:10424000E66EE6EC1BF0E5503A0EE66EE6EC1BF08F
:10425000E550200EE66EE6EC1BF0E550140EE66E1F
:10426000D9CF00F0DACF01F000C0E6FF01C0E6FFD1
:104270004BEC1FF0E550E550E550D9CF00F0DACF18
:1042800001F0140E002600C0E6FF01C0E6FFD9CF02
:1042900002F0DACF03F002C0E6FF03C0E6FF88ECCD
:1042A0001FF0040EE15EF3500BE1370EE66E6E0E6A
:1042B000E66E28EC1FF0E550E5509EBA29D0FDD7F8
:1042C000180EDBCFE9FFE828DBCFEAFFE9CF00F0EB
:1042D000EACF01F0140EDBCF02F0150EDBCF03F0B6
:1042E000160EDBCF04F0170EDBCF05F000C0E9FFA0
:1042F00001C0EAFF02C0EEFF03C0EEFF04C0EEFF04
:1043000005C0EFFF05D00201188102D0020118910B
:104310001B0EE15EE7CFD9FF1200D9CFE6FFE1CF58
:10432000D9FF010EE126E00EE66E6C0EE66E28EC7B
:104330001FF0E550E55050EC20F0F3CF00F000C046
:10434000DFFFDF50390A05E0DF50E66E6CEC20F04D
:10435000E550DF50380AE7E1020EE15EE7CFD9FF12
:1043600012004C0EE66ED7EC39F0E5501200150E37
:10437000E66ED7EC39F0E5501200330EE66EF3EC42
:0643800039F0E5501200C7
:0A4386003C68746D6C3E3C68656194
:10439000643E3C7469746C653E5765622053657277
:1043A00076657220492F4F20436F6E74726F6C3C9C
:1043B0002F7469746C653E3C2F686561643E3C6295
:1043C0006F64793E3C63656E7465723E3C666F6EE9
:1043D0007420666163653D68656C766574696361C8
:1043E0003E3C68323E3C753E4F7574707574204398
:1043F0006F6E74726F6C3C2F753E3C2F68323E3C82
:10440000464F524D204D4554484F443D474554205A
:10441000616374696F6E3D303E3C7461626C65200F
:10442000626F726465723D323E3C74723E3C7464ED
:104430003E3C696E70757420747970653D73756269
:104440006D6974206E616D653D312076616C7565B6
:104450003D44363D2530313E3C2F74643E3C74640F
:104460003E3C696E70757420747970653D73756239
:104470006D6974206E616D653D302076616C756587
:104480003D44353D2530303E3C2F74643E3C2F7416
:10449000723E3C2F7461626C653E3C2F666F726D9C
:1044A0003E3C2F626F64793E3C2F68746D6C3E0415
:1044B000FFFFFF3C48544D4C3E3C484541443E3C88
:1044C0005449544C453E4D6963726F63686970206E
:1044D0005443502F495020537461636B2044656DE1
:1044E0006F3C2F5449544C453E3C2F484541443E77
:1044F0003C4652414D4553455420726F77733D22DF
:104500003130302C33302220626F726465723D305E
:104510003E20203C4652414D45206E616D653D2256
:10452000746F702220097372633D226D61696E2E73
:1045300068746D22206D617267696E68656967686D
:10454000743D35206D617267696E77696474683D8A
:10455000353E093C4652414D4553455420636F6CEE
:10456000733D2238302C38302220626F72646572BD
:104570003D303E202009093C4652414D45206E61A8
:104580006D653D226C656674222020207372633D48
:10459000225374617475732E63676922206D617292
:1045A00067696E6865696768743D32206D6172671E
:1045B000696E77696474683D323E202009093C4683
:1045C00052414D45206E616D653D22726967687488
:1045D000222020207372633D22436F6D6D616E64F3
:1045E000732E63676922206D617267696E68656901
:1045F0006768743D32206D617267696E77696474B3
:10460000683D323E093C2F4652414D455345543E8C
:104610003C2F4652414D455345543E3C2F48544D46
:104620004C3E04FFFFFF3C48544D4C3E3C48454146
:10463000443E3C2F484541443E3C424F44593E3C59
:10464000666F6E7420666163653D68656C7665743F
:104650006963613E3C63656E7465723E3C423E3CFC
:10466000553E3C464F4E542053495A453D37204312
:104670004F4C4F523D2223303030306666223E3C54
:10468000503E4D6963726F63686970205443502FC8
:10469000495020537461636B3C2F503E3C2F423E87
:1046A0003C2F553E3C2F464F4E543E3C2F63656E8B
:1046B0007465723E54686973206973206120736168
:1046C0006D706C65207061676520696E74656E64DD
:1046D000656420746F2064656D6F6E7374726174AD
:1046E00065204D6963726F63686970205443502F71
:1046F000495020537461636B206361706162696C1F
:1047000069746965732E54686973207061676520E8
:104710006973207365727665642062792048545409
:1047200050205365727665722C2072756E6E696EBC
:1047300067206F6E204D6963726F636869702050E7
:1047400049433138206D6963726F636F6E74726FA5
:104750006C6C65722C7574696C697A696E67204D32
:104760006963726F63686970205443502F49502009
:10477000537461636B2E3C703E4D6963726F636866
:10478000697020537461636B206F66666572732075
:10479000666F6C6C6F77696E6720666561747572A1
:1047A00065733A3C2F703E3C756C3E3C6C693E50E4
:1047B0006F727461626C65206163726F7373204DF8
:1047C0006963726F636869702050494331382066AD
:1047D000616D696C79206F66206D6963726F636FBC
:1047E0006E74726F6C6C6572733C2F6C693E3C6CBE
:1047F000693E436F6F7065726174697665206D758F
:104800006C74697461736B696E67205443502F49EF
:104810005020737461636B3C2F6C693E3C6C693E45
:104820005573652069742061732070617274206F04
:1048300066204854545020536572766572206F721A
:1048400020637573746F6D205443502F495020625C
:1048500061736564206170706C69636174696F6E07
:104860003C2F6C693E3C6C693E4D756C7469706C94
:10487000652054435020736F636B657420737570AB
:10488000706F72743C2F6C693E3C6C693E485454A6
:1048900050205365727665722077697468206D7553
:1048A0006C7469706C6520636F6E6E656374696F9C
:1048B0006E7320737570706F72743C2F6C693E3C20
:1048C0006C693E5061676573206D61792062652077
:1048D00073746F72656420696E20696E7465726EA0
:1048E000616C2070726F6772616D206D656D6F72A3
:1048F00079206F722065787465726E616C206461D6
:10490000746120454550524F4D3C2F6C693E3C6CC4
:10491000693E537570706F727420666F72204854D0
:104920004D4C20666F726D733C2F6C693E3C6C6918
:104930003E50432062617365642070726F677261DC
:104940006D20746F20636F6E766572742077656278
:1049500020706167657320696E746F204D696372A2
:104960006F636869702046696C652053797374655C
:104970006D20284D504653293C2F6C693E3C6C6994
:104980003E4D6F64756C61722064657369676E205B
:10499000746F20656173696C7920616464206E6551
:1049A0007720636F6D706F6E656E74733C2F6C69EA
:1049B0003E3C2F756C3E3C2F424F44593E3C2F48A5
:1049C000544D4C3E04FFFFFF3C68746D6C3E3C6DE3
:1049D00065746120687474702D65717569763D2207
:1049E000726566726573682220636F6E74656E749B
:1049F0003D2233223E3C686561643E3C7469746CC0
:104A0000653E576562205365727665722053746106
:104A10007475733C2F7469746C653E3C2F686561D6
:104A2000643E3C626F64793E3C63656E7465723EC1
:104A30003C666F6E7420666163653D68656C766583
:104A4000746963613E3C753E3C68323E53797374D1
:104A5000656D205374617475733C2F68323E3C2F32
:104A6000753E3C7461626C6520626F726465723D74
:104A7000323E3C74723E3C74643E53333D253034C8
:104A80003C2F74643E3C74643E44363D2530313CDA
:104A90002F74643E3C74643E44353D2530303C2FD9
:104AA00074643E3C74643E414E303D2530323C2FB0
:104AB00074643E3C74643E414E313D2530333C2F9E
:104AC00074643E3C2F74723E3C2F7461626C653E90
:104AD0003C62723E3C2F626F64793E3C2F68746D7D
:104AE0006C3E04FFFFFF008643434F4D4D414E4453
:104AF000532E43474900B344494E4445582E485429
:104B00004D2020200026464D41494E2E48544D2030
:104B100020202000C8495354415455532E4347493F
:104B2000202004FFFF454E44204F4620464154209C
:024B3000200063
:0E4B3200D9CFE6FFE1CFD9FF310EE126140EF8
:104B4000E66EE66AD9CF00F0DACF01F0080E002653
:104B500000C0E6FF01C0E6FFEEEC29F0040EE15EC6
:104B6000080EDB50F00B400A01E042D1080EDB508A
:104B70000F0B3F0BE846E846EC0F006E1C0E00C022
:104B8000DBFFDB50140801E233D11C0EDB500008C0
:104B900016E21C0EDBCF00F0016A00C0E6FF01C088
:104BA000E6FFD9CF02F0DACF03F01D0E022602C0D5
:104BB000E6FF03C0E6FFEEEC29F0040EE15E120E04
:104BC000DBCF00F0E828DBCF01F000C0DFFF010EF3
:104BD00001C0DBFF120ED926DE6ADD6AD95E140E33
:104BE000E66EE66AD9CF02F0DACF03F0080E0226AD
:104BF00002C0E6FF03C0E6FF44EC31F0F4CF01F061
:104C0000F3CF00F0040EE15E001E011E00C0DBFFCA
:104C1000050E01C0DBFF1C0EDB50000823E21C0E5A
:104C2000DBCF02F0036A02C0E6FF03C0E6FFD9CF84
:104C300004F0DACF05F01D0E042604C0E6FF05C01F
:104C4000E6FF44EC31F0F4CF01F0F3CF00F0040EB6
:104C5000E15E001E011E060E00C0DBFF070E01C054
:104C6000DBFF05D0060ED926DE6ADD6AD95E040EAA
:104C7000E66EE66AD9CF02F0DACF03F0022602C070
:104C8000E6FF03C0E6FF44EC31F0F4CF01F0F3CFD0
:104C900000F0040EE15E020E00C0DBFF030E01C057
:104CA000DBFFD9CF00F0DACF01F0080E002600C0FC
:104CB000E6FF01C0E6FFBEEC27F0E550E550000E30
:104CC000DBCF00F0E828DBCF01F0020EDBCF02F0F3
:104CD000E828DBCF03F00050025C07E101500358E5
:104CE00004E1080EDB50F00B400A01E081D0D9CF7F
:104CF000E9FFDACFEAFFFD0EE926EE5001E1ED50C3
:104D000022E0FD0EDBCFE9FFE828DBCFEAFFE9CFA9
:104D100000F0EACF01F0180EDBCF02F0190EDBCF66
:104D200003F01A0EDBCF04F01B0EDBCF05F000C042
:104D3000E9FF01C0EAFF02C0EEFF03C0EEFF04C0BE
:104D4000EEFF05C0EFFFFB0EDBCFE9FFE828DBCF6E
:104D5000EAFF060EE926000EEA22E9CF00F0EACFCC
:104D600001F0140EDBCF02F0150EDBCF03F0160EB0
:104D7000DBCF04F0170EDBCF05F000C0E9FF01C068
:104D8000EAFF02C0EEFF03C0EEFF04C0EEFF05C065
:104D9000EFFFF90EDBCF00F0E828DBCF01F0110EBA
:104DA000DB5000C0E9FF01C0EAFFEF6EF70EDBCF7A
:104DB00000F0E828DBCF01F00A0EDBCF04F0E82892
:104DC000DBCF05F01C0EDB50045C026E0550036A5D
:104DD0000356140E025E000E035A00C0E9FF01C024
:104DE000EAFF02C0EEFF03C0EDFF010EF36E03D039
:104DF00024EC2AF0F36A320EE15EE7CFD9FF12000D
:104E0000D9CFE6FFE1CFD9FF140EE126450EDF6EC4
:104E1000010EDB6AFA0EDBCF00F0E828DBCF01F0F1
:104E2000140E0026000E0122020E00C0DBFF030E4E
:104E300001C0DBFF0101FE4BFF2B040EFEC1DBFFB7
:104E4000050EFFC1DBFF060ED926DE6ADD6AD95EDC
:104E5000640EE76E080EE7CFDBFFFC0EDBCF00F041
:104E6000090E00C0DBFF0A0ED926DE6ADD6AD95EB4
:104E70000C0E00C2DBFF0D0E01C2DBFF0E0E02C2E4
:104E8000DBFF0F0E03C2DBFFFD0EDBCFE9FFE828DF
:104E9000DBCFEAFF060EE926000EEA22EECF00F095
:104EA000EECF01F0EECF02F0EECF03F0100E00C017
:104EB000DBFF110E01C0DBFF120E02C0DBFF130E81
:104EC00003C0DBFFD9CF00F0DACF01F000C0E6FF6E
:104ED00001C0E6FFBEEC27F0E550E550140EE66E8B
:104EE000E66AD9CF02F0DACF03F002C0E6FF03C0D2
:104EF000E6FF44EC31F0F4CF01F0F3CF00F0040E04
:104F0000E15E0A0E00C0DBFF0B0E01C0DBFFFA0EF4
:104F1000DBCF00F0E828DBCF01F0140E0026000EF6
:104F2000012200C0E6FF01C0E6FFE66AFD0EDBCF0E
:104F3000E9FFE828DBCFEAFFE9CF02F0EACF03F090
:104F400002C0E6FF03C0E6FF37EC2AF0050EE15E83
:104F5000140EE66EE66AD9CF00F0DACF01F000C099
:104F6000E6FF01C0E6FF81EC2AF0040EE15EF36A81
:104F7000F46A150EE15EE7CFD9FF1200D9CFE6FF44
:104F8000E1CFD9FFFD0EDBCFE9FFE828DBCFEAFF59
:104F9000EE52EE52E9CF00F0EACF01F000C0E6FF9A
:104FA00001C0E6FFFD0EDBCFE9FFE828DBCFEAFF1B
:104FB000EE52EE52EECF04F0EECF05F004C0E6FF65
:104FC00005C0E6FF5EEC30F0F4CF03F0F3CF02F063
:104FD000E550E550E550E5CF01F0E7CF00F000C027
:104FE000E9FF01C0EAFF02C0EEFF03C0EDFFFD0EC6
:104FF000DBCFE9FFE828DBCFEAFF040EE926000E4D
:10500000EA22E9CF00F0EACF01F000C0E6FF01C0DC
:10501000E6FFFD0EDBCFE9FFE828DBCFEAFF040E59
:10502000E926000EEA22EECF04F0EECF05F004C030
:10503000E6FF05C0E6FF5EEC30F0F4CF03F0F3CFFF
:1050400002F0E550E550E550E5CF01F0E7CF00F084
:1050500000C0E9FF01C0EAFF02C0EEFF03C0EDFFA0
:10506000FD0EDBCFE9FFE828DBCFEAFF0A0EE926D9
:10507000000EEA22E9CF00F0EACF01F000C0E6FF1F
:1050800001C0E6FFFD0EDBCFE9FFE828DBCFEAFF3A
:105090000A0EE926000EEA22EECF04F0EECF05F06C
:1050A00004C0E6FF05C0E6FF5EEC30F0F4CF03F08D
:1050B000F3CF02F0E550E550E550E5CF01F0E7CF42
:1050C00000F000C0E9FF01C0EAFF02C0EEFF03C02C
:0A50D000EDFFE552E7CFD9FF120013
:0650DA009EAA8FD09DAAE2
:1050E0008DD0AB50060B05E0AB98AB880201050EE6
:1050F000346FAECF32F2020136913451050A47E0E7
:10510000010A35E0070A22E0010A18E0030A10E06C
:1051100002C333F2356BC00E326303D0030E346F1B
:1051200039D0410E326336D03681020E346F32D020
:1051300036810D0E32632ED036832CD03681540E3C
:10514000326302D0010E08D0050E06D03681DB0E88
:10515000326304D03691040E346F1CD0C00E32631B
:1051600019D0355102E0368315D0369113D03681EF
:10517000030E346FDC0E326302D0C00E04D0DD0E9D
:10518000326303D0DB0E326F05D0369102D033C2CA
:1051900002F3346B36A11ED00301022BFA0E025D1E
:1051A00001E3026B0251005D10E00201352B040E99
:1051B000006E030E016E03010251EA6A0024E96EDB
:1051C0000150EA2232C2EFFF05D033C202F30201DE
:1051D000346B3693020136A311D03693040E006E61
:1051E000030E016E3351EA6A0024E96E0150EA228F
:1051F00002C3EFFF0301012B0201346B9EA845D0CF
:105200009DA843D00401005139E0040E006E040E45
:10521000016E0151EA6A0024E96E0150EA22EECFE4
:1052200032F2C00E0201326310D0DB0E326F040E78
:10523000006E040E016E04010151EA6A0024E96E59
:105240000150EA22DC0EEF6E16D0DB0E326310D076
:10525000DB0E326F040E006E040E016E040101516C
:10526000EA6A0024E96E0150EA22DD0EEF6E03D0F7
:1052700004010007012B32C2ADFF07D09D9803A1A6
:1052800002D0039102D0C00EAD6E1200E66AAEEC01
:105290002AF0E5500201346B366B0301006B016BA1
:1052A000036B026B0201316B9E9A9D8A9D98200EC2
:1052B000AC6E900EAB6E070EAF6EF28EF28C1200DB
:1052C000FA0E0401005D01E304D09DB802D0010E86
:1052D00001D0000EF36E1200D9CFE6FFE1CFD9FF67
:1052E0000201010E316F030101513EE000C303F3DF
:1052F000032BFA0E035D01E3036B040E006E030E35
:10530000016E0351EA6A0024E96E0150EA22EF506F
:10531000410A20E124EC2AF004010381040E006F0D
:10532000026B0201316B4F0EE66E4BEC2AF0E5503A
:105330004B0EE66E4BEC2AF0E5500D0EE66E4BEC94
:105340002AF0E5500A0EE66E4BEC2AF0E550A5EC8B
:105350002AF00AD0FB0EDBCFE9FFE828DBCFEAFF1B
:10536000EF6A010EF36E01D0F36AE552E7CFD9FF81
:105370001200D9CFE6FFE1CFD9FF010EE1260201ED
:10538000315115E0040E016E030E026E030103514C
:10539000032BEA6A0124E96E0250EA22EECF00F004
:1053A00000C0DFFFFA0E035D12E3036B10D0040EA2
:1053B000016E040E026E04010251022BEA6A0124FE
:1053C000E96E0250EA22EECF00F000C0DFFFDF50AE
:1053D000F36E020EE15EE7CFD9FF1200D9CFE6FFF0
:1053E000E1CFD9FFFB0EDBCF00F0DB06FC0EDBCFFD
:1053F00001F001E2DB06005001E101501BE0FD0E6F
:10540000DBCF00F0DB2AFE0EDBCF01F001E1DB2A6F
:1054100000C0E6FF01C0E6FFB9EC29F0E550E5CF9A
:1054200001F0E7CF00F0F35000C0E9FF01C0EAFF50
:10543000EF6ED8D7FB0EDBCFF3FFE828DBCFF4FF0E
:10544000E552E7CFD9FF12009D9A030101510DE00B
:10545000040E006E030E016E0051EA6A0024E96E2C
:105460000150EA22EECF00F301079D8A1200D9CF46
:10547000E6FFE1CFD9FFD9CFE9FFDACFEAFFFA0E95
:10548000E926EECF00F40401026B0201316BE55214
:10549000E7CFD9FF1200D9CFE6FFE1CFD9FF020154
:1054A000315118E0040E026E030E036E0301035126
:1054B000032B016A0224006E03500122FE0EDB5012
:1054C00000C0E9FF01C0EAFFEF6EFA0E035D15E3CD
:1054D000036B13D0040E026E040E036E040102511E
:1054E000022B016A0224006E03500122FE0EDB50E3
:1054F00000C0E9FF01C0EAFFEF6EE552E7CFD9FF38
:105500001200D9CFE6FFE1CFD9FFFB0EDBCF00F0D1
:10551000DB06FC0EDBCF01F001E2DB06005001E10F
:1055200001500FE0FD0EDBCFE9FFDB2AFE0EDBCFE3
:10553000EAFF01E1DB2AEF50E66E4BEC2AF0E55082
:10554000E4D7E552E7CFD9FF12000401026B016BEB
:1055500003B102D0C00EAD6E9D881200D9CFE6FF18
:10556000E1CFD9FF9DB805D00401006B026B016B40
:10557000036BE552E7CFD9FF1200D9CFE6FFE1CFA9
:10558000D9FFD9CF00F0DACF01F0FD0E002600C31D
:1055900002F0036A00C0E9FF01C0EAFF0250EE26F4
:1055A0000350ED22FD0EDB2A02E1FE0EDB2AFD0E8A
:1055B000DBCF00F0E828DBCF01F0F90E005C000E35
:1055C00001580DE3FD0EDBCF00F0E828DBCF01F042
:1055D000FA0E005E000E015A00C003F308D0D9CFC6
:1055E000E9FFDACFEAFFFD0EE926EECF03F3020171
:1055F000010E316FE552E7CFD9FF1200D9CFE6FF98
:10560000E1CFD9FFD9CFE9FFDACFEAFFFC0EE926D7
:10561000EECF02F40201316BE552E7CFD9FF120061
:10562000D9CFE6FFE1CFD9FFE552E7CFD9FF12008E
:10563000D9CFE6FFE1CFD9FF010EE1269D9A02C343
:10564000DFFF9D8A030101510DE0DFCF00F0005123
:10565000D880005404E2DF50FA08002504D0DF505F
:10566000005D01D0F80EF36EF46A020EE15EE7CF42
:04567000D9FF12004C
:0C567400D9CFE6FFE1CFD9FF1C0EE126E4
:10568000E66EE66AD9CF00F0DACF01F000C0E6FF9F
:1056900001C0E6FFEEEC29F0040EE15E24EC2AF0F6
:1056A000D9CF00F0DACF01F000C0E6FF01C0E6FF7D
:1056B00053EC2DF0E550E550000EDBCF00F0E8286C
:1056C000DBCF01F0010E005C13E1015811E1040E83
:1056D000DBCF02F0036A060E025C0AE1035808E120
:1056E000050EDBCF04F0056A040E045C01E10558E9
:1056F00001E09AD0060EDBCF00F0E828DBCF01F006
:10570000020E005C0AE1015808E1FB0EDBCFE9FF65
:10571000E828DBCFEAFFEF6A1DD0060EDBCF00F0F2
:10572000E828DBCF01F0010E005C0BE1015809E134
:10573000FB0EDBCFE9FFE828DBCFEAFF010EEF6EBF
:1057400009D0FB0EDBCFE9FFE828DBCFEAFF020E32
:10575000EF6E6AD0180EDB500201005D01E064D0EC
:10576000190EDB50015D01E05FD01A0EDB50025DC7
:1057700001E05AD01B0EDB50035D01E055D0FD0E59
:10578000DBCFE9FFE828DBCFEAFFE9CF00F0EACF83
:1057900001F0080EDBCF02F0090EDBCF03F00A0E9A
:1057A000DBCF04F00B0EDBCF05F00C0EDBCF06F0E9
:1057B0000D0EDBCF07F000C0E9FF01C0EAFF02C019
:1057C000EEFF03C0EEFF04C0EEFF05C0EEFF06C013
:1057D000EEFF07C0EFFFFD0EDBCFE9FFE828DBCFD0
:1057E000EAFF060EE926000EEA22E9CF00F0EACF32
:1057F00001F00E0EDBCF02F00F0EDBCF03F0100E28
:10580000DBCF04F0110EDBCF05F000C0E9FF01C0D3
:10581000EAFF02C0EEFF03C0EEFF04C0EEFF05C0CA
:10582000EFFF010EF36E01D0F36A1D0EE15EE7CFCC
:10583000D9FF1200D9CFE6FFE1CFD9FF1C0EE12638
:10584000010EDE6EDD6A020ED926DE6A080EDD6EFE
:10585000020ED95E060EE76E040EE7CFDBFFE76EA1
:10586000050EE7CFDBFFFC0EDB50010A14E1060E4C
:10587000D926010EDE6EDD6A060ED95E120EDB68D9
:10588000130EDB68140EDB68150EDB68160EDB6882
:10589000170EDB6833D0060ED926020EDE6EDD6AE7
:1058A000060ED95EFD0EDBCFE9FFE828DBCFEAFF6D
:1058B000EECF00F0EECF01F0EECF02F0EECF03F02E
:1058C000EECF04F0EECF05F0EECF06F0EECF07F00E
:1058D000EECF08F0EECF09F0120E00C0DBFF130E82
:1058E00001C0DBFF140E02C0DBFF150E03C0DBFF9F
:1058F000160E04C0DBFF170E05C0DBFF080E04C246
:10590000DBFF090E05C2DBFF0A0E06C2DBFF0B0E32
:1059100007C2DBFF0C0E08C2DBFF0D0E09C2DBFF66
:105920000E0E00C2DBFF0F0E01C2DBFF100E02C223
:10593000DBFF110E03C2DBFF0E0EDBCF01F0FD0E0D
:10594000DBCFE9FFE828DBCFEAFF060EE926000EF1
:10595000EA22EF500118006E02010A510014E850CB
:1059600041E10F0EDBCF03F0FD0EDBCFE9FFE828AE
:10597000DBCFEAFF060EE926000EEA22EE52EF50D8
:105980000318026E0B510214E8502CE1100EDBCF0D
:1059900005F0FD0EDBCFE9FFE828DBCFEAFF060EBE
:1059A000E926000EEA22EE52EE52EF500518046E80
:1059B0000C510414E85016E1110EDBCF07F0FD0E78
:1059C000DBCFE9FFE828DBCFEAFF060EE926000E71
:1059D000EA22EE52EE52EE52EF500718066E0D51CB
:1059E0000614E8500DE0180E0EC2DBFF190E0FC2B0
:1059F000DBFF1A0E10C2DBFF1B0E11C2DBFF1ED035
:105A0000FD0EDBCFE9FFE828DBCFEAFF060EE92633
:105A1000000EEA22EECF00F0EECF01F0EECF02F062
:105A2000EECF03F0180E00C0DBFF190E01C0DBFF44
:105A30001A0E02C0DBFF1B0E03C0DBFFD9CF00F044
:105A4000DACF01F000C0E6FF01C0E6FF53EC2DF015
:105A5000E550E5501C0EE66EE66A060EE66ED9CFFE
:105A600000F0DACF01F0120E002600C0E6FF01C000
:105A7000E6FF37EC2AF0050EE15E1C0EE66EE66AE4
:105A8000D9CF00F0DACF01F000C0E6FF01C0E6FF99
:105A900081EC2AF0040EE15EA5EC2AF01D0EE15E19
:105AA000E7CFD9FF1200D9CFE6FFE1CFD9FFFD0E36
:105AB000DBCFE9FFE828DBCFEAFFE9CF00F0EACF50
:105AC00001F000C0E6FF01C0E6FFFD0EDBCFE9FFFD
:105AD000E828DBCFEAFFEECF04F0EECF05F004C0FC
:105AE000E6FF05C0E6FF5EEC30F0F4CF03F0F3CF45
:105AF00002F0E550E550E550E5CF01F0E7CF00F0CA
:105B000000C0E9FF01C0EAFF02C0EEFF03C0EDFFE5
:105B1000FD0EDBCFE9FFE828DBCFEAFFEE52EE52C5
:105B2000E9CF00F0EACF01F000C0E6FF01C0E6FFD8
:105B3000FD0EDBCFE9FFE828DBCFEAFFEE52EE52A5
:105B4000EECF04F0EECF05F004C0E6FF05C0E6FF9F
:105B50005EEC30F0F4CF03F0F3CF02F0E550E55007
:105B6000E550E5CF01F0E7CF00F000C0E9FF01C04C
:105B7000EAFF02C0EEFF03C0EDFFFD0EDBCFE9FF41
:105B8000E828DBCFEAFF060EE926000EEA22E9CF7D
:105B900000F0EACF01F000C0E6FF01C0E6FFFD0E15
:105BA000DBCFE9FFE828DBCFEAFF060EE926000E8F
:105BB000EA22EECF04F0EECF05F004C0E6FF05C008
:105BC000E6FF5EEC30F0F4CF03F0F3CF02F0E550E7
:105BD000E550E550E5CF01F0E7CF00F000C0E9FF68
:105BE00001C0EAFF02C0EEFF03C0EDFFE552E7CFC0
:045BF000D9FF1200C7
:0C5BF400D9CFE6FFE1CFD9FF300EE1264B
:105C0000080EE66EE66AD9CF00F0DACF01F000C0E8
:105C1000E6FF01C0E6FFEEEC29F0040EE15E020EA5
:105C2000DBCF00F0E828DBCF01F02E0E00C0DBFF59
:105C30002F0E01C0DBFF020ED926DE6ADD6AD95EB7
:105C4000080EE66EE66AD9CF02F0DACF03F002C0A2
:105C5000E6FF03C0E6FF44EC31F0F4CF01F0F3CFF0
:105C600000F0040EE15E001E011E280E00C0DBFFE6
:105C7000290E01C0DBFFF90EDBCFE9FFE828DBCFFF
:105C8000EAFF080EEF5EF90EDBCFE9FFE828DBCF75
:105C9000EAFFEECF00F0016A00C0E6FF01C0E6FFB8
:105CA000FB0EDBCF02F0E828DBCF03F002C0E6FFFB
:105CB00003C0E6FFEEEC29F0040EE15EF90EDBCF47
:105CC000E9FFE828DBCFEAFFEECF02F0036A02C06B
:105CD000E6FF03C0E6FFFB0EDBCF04F0E828DBCFD6
:105CE00005F004C0E6FF05C0E6FF44EC31F0F4CF58
:105CF00001F0F3CF00F0040EE15E001E011E2A0E3B
:105D000000C0DBFF2B0E01C0DBFF040EE66EE66A6F
:105D1000D9CF02F0DACF03F0280E022602C0E6FF48
:105D200003C0E6FF44EC31F0F4CF01F0F3CF00F014
:105D3000040EE15E2C0E00C0DBFF2D0E01C0DBFF68
:105D4000D9CF00F0DACF01F000C0E6FF01C0E6FFD6
:105D5000AFEC2FF0E550E550FD0EDBCF00F0E8286A
:105D6000DBCF01F0DF5000C0E9FF01C0EAFFEF6EBA
:105D7000F70EDBCF00F0E828DBCF01F0040EDBCF1D
:105D800002F0E828DBCF03F000C0E9FF01C0EAFF22
:105D900002C0EEFF03C0EDFFF50EDBCF00F0E828F8
:105DA000DBCF01F0060EDBCF02F0E828DBCF03F0FB
:105DB00000C0E9FF01C0EAFF02C0EEFF03C0EDFF33
:105DC0002C0EDBCF00F0E828DBCF01F02E0EDBCF6E
:105DD00002F0E828DBCF03F00050025C04E1015040
:105DE000035801E102D0000E01D0010EF36E310E16
:105DF000E15EE7CFD9FF1200D9CFE6FFE1CFD9FFAF
:105E0000280EE126010EDB6AFC0EDBCF00F000C09D
:105E1000DFFF020ED926DE6ADD6AD95EF70EDBCF20
:105E200000F0E828DBCF01F0040E00C0DBFF050E18
:105E300001C0DBFFF50EDBCF00F0E828DBCF01F07F
:105E4000060E00C0DBFF070E01C0DBFFF90EDBCF43
:105E500000F0016A00C0E6FF01C0E6FFFA0EDBCFEA
:105E600002F0E828DBCF03F002C0E6FF03C0E6FF44
:105E7000D9CF04F0DACF05F0080E042604C0E6FFFF
:105E800005C0E6FF61EC37F0060EE15ED9CF00F009
:105E9000DACF01F000C0E6FF01C0E6FFAFEC2FF063
:105EA000E550E550F90EDBCF02F0036A080E02263A
:105EB000000E032202C0E6FF03C0E6FFD9CF04F0C4
:105EC000DACF05F004C0E6FF05C0E6FF44EC31F090
:105ED000F4CF01F0F3CF00F0040EE15E020E00C03B
:105EE000DBFF030E01C0DBFFF90EDBCF00F0016A20
:105EF000080E0026000E012200C0E6FF01C0E6FFEA
:105F0000010EE66EFD0EDBCF02F0E828DBCF03F0DA
:105F100002C0E6FF03C0E6FF00EC27F0050EE15EDD
:105F2000F90EDBCF00F0016A080E0026000E0122F8
:105F300000C0E6FF01C0E6FFD9CF02F0DACF03F0E0
:105F400002C0E6FF03C0E6FF81EC2AF0040EE15E2A
:105F5000A5EC2AF0290EE15EE7CFD9FF1200D9CFD8
:105F6000E6FFE1CFD9FFFD0EDBCFE9FFE828DBCF6D
:105F7000EAFF040EE926000EEA22E9CF00F0EACF9C
:105F800001F000C0E6FF01C0E6FFFD0EDBCFE9FF38
:105F9000E828DBCFEAFF040EE926000EEA22EECF66
:105FA00004F0EECF05F004C0E6FF05C0E6FF5EECAE
:105FB00030F0F4CF03F0F3CF02F0E550E550E550B8
:105FC000E5CF01F0E7CF00F000C0E9FF01C0EAFF34
:105FD00002C0EEFF03C0EDFFFD0EDBCFE9FFE828B6
:105FE000DBCFEAFF060EE926000EEA22E9CF00F039
:105FF000EACF01F000C0E6FF01C0E6FFFD0EDBCFF7
:10600000E9FFE828DBCFEAFF060EE926000EEA22C8
:10601000EECF04F0EECF05F004C0E6FF05C0E6FFCA
:106020005EEC30F0F4CF03F0F3CF02F0E550E55032
:10603000E550E5CF01F0E7CF00F000C0E9FF01C077
:10604000EAFF02C0EEFF03C0EDFFFD0EDBCFE9FF6C
:10605000E828DBCFEAFFEE52EE52E9CF00F0EACFBC
:1060600001F000C0E6FF01C0E6FFFD0EDBCFE9FF57
:10607000E828DBCFEAFFEE52EE52EECF04F0EECF8F
:1060800005F004C0E6FF05C0E6FF5EEC30F0F4CF9B
:1060900003F0F3CF02F0E550E550E550E5CF01F015
:1060A000E7CF00F000C0E9FF01C0EAFF02C0EEFF49
:0C60B00003C0EDFFE552E7CFD9FF12005E
:0460BC00D9CFE6FF53
:1060C000E1CFD9FF030EE126FD0EDBCF00F0E8287B
:1060D000DBCF01F000C0DFFF010E01C0DBFFDBCF33
:1060E00000F0020E00C0DBFFDFCF00F0010E00C0A9
:1060F000DBFF020EDBCF00F000C0DFFF000EDBCFC6
:10610000F3FFE828DBCFF4FF040EE15EE7CFD9FF11
:106110001200D9CFE6FFE1CFD9FF070EE126FB0E33
:10612000DBCF00F0FC0EDBCF01F0FD0EDBCF02F089
:10613000FE0EDBCF03F0010E00C0DBFF020E01C03C
:10614000DBFF030E02C0DBFF040E03C0DBFFD9CF71
:1061500000F0DACF01F0010E0026050E00C0DBFFD3
:10616000060E01C0DBFF050EDBCFE9FFE828DBCF21
:10617000EAFFEE52EE52EE52EECF00F000C0DFFF2B
:10618000050EDBCFE9FFE828DBCFEAFFE9CF00F01F
:10619000EACF01F0030E0026000E0122050EDBCF30
:1061A000E9FFE828DBCFEAFFEF5000C0E9FF01C0BC
:1061B000EAFFEF6E050EDBCFE9FFE828DBCFEAFF51
:1061C000E9CF00F0EACF01F0DF5000C0E9FF01C0E5
:1061D000EAFFEF6E050EDBCFE9FFE828DBCFEAFF31
:1061E000EE52EE52EECF00F000C0DFFF050EDBCF27
:1061F000E9FFE828DBCFEAFFE9CF00F0EACF01F0C2
:10620000020E0026000E0122050EDBCFE9FFE82872
:10621000DBCFEAFFEE52EF5000C0E9FF01C0EAFF1A
:10622000EF6E050EDBCFE9FFE828DBCFEAFFE9CF11
:1062300000F0EACF01F0010E0026000E0122DF502F
:1062400000C0E9FF01C0EAFFEF6E010EDBCF00F0F6
:10625000020EDBCF01F0030EDBCF02F0040EDBCF2A
:1062600003F0020ED95CE96E000EDA58EA6E03C044
:10627000EDFF02C0EDFF01C0EDFF00C0EFFF080E13
:10628000E15EE7CFD9FF1200D9CFE6FFE1CFD9FF1A
:106290000A0EE126DE6ADE6ADE6ADD6ADD52DD5262
:1062A000FB0EDBCF02F0E828DBCF03F002C000F0EA
:1062B00003C001F0D89001320032040E00C0DBFFB1
:1062C000050E01C0DBFFFD0EDBCF00F0E828DBCFC1
:1062D00001F0060E00C0DBFF070E01C0DBFF040E5D
:1062E000DBCF00F0DB06050EDBCF01F001E2DB06C1
:1062F000005001E1015020E0D9CF00F0DACF01F0E9
:10630000060ED926DECFE9FFDDCFEAFF020EDE263C
:10631000000EDD22060ED95EEECF02F0EECF03F0C6
:1063200000C0E9FF01C0EAFF0250EE260350EE2252
:10633000000EEE22EE22D3D7FB0EDBCF00F0E828D2
:10634000DBCF01F00050010B16E0D9CF00F0DACF1F
:1063500001F0060EDBCFE9FFE828DBCFEAFFEECF46
:1063600002F000C0E9FF01C0EAFF0250EE26000E75
:10637000EE22EE22EE22D9CFE9FFDACFEAFFEC508F
:10638000ECCF02F0ECCF03F0046A056A02C000F023
:1063900003C001F0080E00C0DBFF090E01C0DBFFE7
:1063A000005001E101502CE0DECF04F0DDCF05F01C
:1063B000020EDBCF06F0030EDBCF07F0066A076A9A
:1063C000080EDBCF08F0E828DBCF09F000010A6BEC
:1063D0000B6B08500424006E09500520016E0A5012
:1063E0000620026E0B500720036E00C0DEFF01C0C6
:1063F000DDFF020E02C0DBFF030E03C0DBFFBBD7D5
:10640000D9CFE9FFDACFEAFFEECFF3FFEECFF4FF0B
:0E641000F31EF41E0B0EE15EE7CFD9FF120063
:02641E00020179
:10642000386B376B010EF36E1200D9CFE6FFE1CF68
:10643000D9FF120EE126020137A103D0F36AF46AF4
:10644000B8D0D9CFE9FFDACFEAFF0F0EE926E60E82
:10645000EE6E4A0EED6EFD0EDBCFE9FFE828DBCFD6
:10646000EAFFEF5001E1A3D0FD0EDBCF02F0E828F8
:10647000DBCF03F002C0E6FF03C0E6FFE7EC37F036
:10648000F4CF01F0F3CF00F0E550E550FD0E00C071
:10649000DBFFFE0E01C0DBFF0F0EE66EE66ADBCF10
:1064A00000F0E828DBCF01F00001026B00C0E6FF3E
:1064B00001C0E6FF02C0E6FFD9CF03F0DACF04F057
:1064C00003C0E6FF04C0E6FF8CEC37F0070EE15E88
:1064D000DF50E86652D0FD0EDBCF02F0E828DBCFBC
:1064E00003F002C0E6FF03C0E6FFAFEC37F0F4CFE5
:1064F00001F0F3CF00F0E550E550110E00C0DBFFD6
:10650000DB500C0805E20C0EE76E110EE7CFDBFF47
:10651000110EDBCF00F0016A00C0E6FF01C0E6FF0C
:10652000D9CF02F0DACF03F0030E022602C0E6FF55
:1065300003C0E6FFFD0EDBCF04F0E828DBCF05F05B
:1065400004C0E6FF05C0E6FFBDEC37F0060EE15ED5
:10655000F35009E10201382B010EDBCFF3FFE828ED
:10656000DBCFF4FF26D0D9CFE9FFDACFEAFF0F0E59
:10657000E926EE26000EED228FD7DF50040A17E140
:10658000010EDBCF00F0E828DBCF01F0FF0E005C4E
:1065900002E1FF0E01580BE0010EDBCF00F0E8280E
:1065A000DBCF01F00F0E00C0DBFF100E73D7F368D6
:1065B000F468130EE15EE7CFD9FF120002013B6BD6
:1065C0003791385101E038071200D9CFE6FFE1CF0B
:1065D000D9FF010EE12639C2F6FF3AC2F7FF0A00E1
:1065E000F5CF00F000C0DFFF0201394B3A2BDF503E
:1065F000030A0CE139C2F6FF3AC2F7FF0A00F5CFF1
:1066000000F000C0DFFF394B3A2B05D0DF50040A01
:1066100002E139693A69DF50F36E020EE15EE7CFBD
:10662000D9FF120002013781200EF36EF46A1200C6
:10663000D9CFE6FFE1CFD9FF010EF36EE552E7CFE8
:0E664000D9FF120039C2F3FF3AC2F4FF120074
:02664E00FF0E3D
:10665000E3CFEAFFE552FF0EE3CFE9FFE552E66A3A
:10666000E66AD9CFE6FFDACFE6FFFC0EE124D96E69
:10667000FF0EE220DA6EE66AE66AE66A200EEF5C5A
:1066800006E0090EEF5C03E0EF6603D03FD0EE506A
:10669000F5D72D0EEF5C03E1FF0EE32A03D02B0E9E
:1066A000EF5C01E1EE502F0EEF6424D03A0EEF6064
:1066B00021D0D890F90EE336FA0EE336FD0EDECF88
:1066C000E3FFFE0EDDCFE3FFD890F90EE336FA0EBE
:1066D000E336D890F90EE336FA0EE336FD0EE350BA
:1066E000DE26FE0EE350DD22300EEE5CDE26000ECE
:1066F000DD22D9D7FF0EE3CFE8FFE85207E0F90E1D
:10670000E31EE32AFA0ED8B4E306E31EE552E5528F
:10671000E552FF0EE3CFDAFFE552FF0EE3CFD9FFDC
:10672000E552E1CFE9FFE2CFEAFFED52ED52EECFC5
:10673000F3FFEFCFF4FF1200D9CFE6FFDACFE6FF89
:10674000FA0EE3CFD9FFFB0EE3CFDAFFFD0EE352E3
:1067500009E72D0EDE6EFC0EE31EE32AFD0ED8B413
:10676000E306E31EE652E652E652FD0EE124E76E32
:10677000FF0EE220E46EE652F70EE3CFE6FFF70EDF
:10678000E3CFE6FF0CEC34F0F90EE124E96EFF0EE6
:10679000E220EA6EFCEC33F00AE1F9EC33F009E1B7
:1067A000FCEC33F008E1F9EC33F007E108D007EC3A
:1067B00034F002EC34F007EC34F002EC34F007EC87
:1067C00034F0DE6AF90EE126FF0EE222FF0EE3CF7F
:1067D000DAFFE552FF0EE3CFD9FFE552FC0EE124CC
:1067E000E96EFF0EE220EA6EEECFF3FFEFCFF4FF8B
:1067F0001200EF380F0B1200EF500F0B02E1EE52B8
:10680000D8841200EF380F0B300FDE6E1200EE50FE
:106810000F0B300FDE6E1200FC0EE3CFE9FFFD0E12
:10682000E3CFEAFF100EE66EEE6AEE6AEF6AD890EA
:10683000FD0EE336FE0EE336ED36ED36EF36FF0E97
:10684000E30609E02DEC34F0EE522DEC34F0EE527C
:106850002DEC34F0EDD7E56E1200030EEF24E8B610
:0C686000EF6E300EEF24E8BEEF6E000C6F
:04686C000001B26B0A
:1068700046EC29F06EEC39F088EC00F01200D9CF2C
:10688000E6FFE1CFD9FF060EE126010EE76E050E09
:10689000E7CFDBFF050EDB5001E1EDD0050EDB6A33
:1068A0000001B251040A01E1C7D0070A01E18CD00E
:1068B000050A01E176D0040A3BE0070A32E0050A46
:1068C00003E0010A01E0E6D7D9CF00F0DACF01F00A
:1068D000040E002600C0E6FF01C0E6FFB30E026E04
:1068E000000E036E02C0E6FF03C0E6FF6CEC29F069
:1068F000040EE15EF35001E1CDD7010EE76E050E07
:10690000E7CFDBFF040EDB50E86603D00001020E88
:1069100041D0040EDB50060A01E08BD00001050EC9
:1069200039D0050EDB6A71EC39F0F350B3E0A0D03A
:10693000BD0EE66E000EE66ED9CF00F0DACF01F0A4
:10694000040E002600C0E6FF01C0E6FFB30EE66EAF
:10695000000EE66ED9CF02F0DACF03F002C0E6FFF8
:1069600003C0E6FF99EC25F0080EE15EF35016E057
:10697000010EE76E050EE7CFDBFF040EDB50010AC8
:1069800003E10001030E06D0040EDB50060A04E109
:106990000001060EB26F7ED7050EDB6A24EC2AF0EA
:1069A00067D0BDC0E6FFBEC0E6FFB30EE66E000EC8
:1069B000E66E19EC06F0040EE15EF35002E0000111
:1069C000B26B050EDB6A66D7B26BBD512908000EAB
:1069D000BE552FE3E10EE66E000EE66EDF0EE66EAC
:1069E000000EE66EBD0EE66E000EE66EBF0EE66EA3
:1069F000000EE66ED9CF00F0DACF01F0040E0026CB
:106A000000C0E6FF01C0E6FFFAEC2DF00A0EE15EE1
:106A1000F3500DE0040EDB50080A09E1010EE76EA9
:106A2000050EE7CFDBFF0001040EB26F02D00001BC
:106A3000B26B24EC2AF02ED760EC29F0F35001E180
:106A400029D7E1C0E6FFE2C0E6FFDFC0E6FFE0C015
:106A5000E6FFBDC0E6FFBF0EE66E000EE66EE66A1C
:106A6000B30EE66E000EE66EFCEC2EF00A0EE15E52
:106A70000001B26B0FD718EC06F0070EE15EE7CF0E
:046A8000D9FF120028
:0C6A8400F00E83160F0E9512959A95984F
:106A9000929A839A8398809AB1EC21F0F00E951621
:106AA00083168382808ABDEC21F0809AB7EC21F0B6
:106AB000F00E83168382808ABDEC21F0809ABDECB3
:106AC00021F0F00E83168382808ABDEC21F0809A3B
:106AD0000F0E9512280EE66E89EC35F0E550080E83
:106AE000E66E89EC35F0E5500C0EE66E89EC35F07B
:106AF000E550010EE66E89EC35F0E550130EE66EBA
:106B000089EC35F0E550800EE66E89EC35F0E55005
:106B10001200D9CFE6FFE1CFD9FFB6EC35F0F35044
:106B200001E0FBD7959A9598F00E95168316FE0E08
:106B3000DB50F00BE83A8312839A8398BDEC21F086
:106B4000808ABDEC21F0809AF00E8316FE0EDB5099
:106B50000F0B8312BDEC21F0808ABDEC21F0809AEE
:106B60000F0E9512E552E7CFD9FF1200959A95982E
:106B7000838A8398BDEC21F0808ABDEC21F083A646
:106B80000BD0809ABDEC21F0808ABDEC21F0809A78
:106B9000839A010EF36E09D0809ABDEC21F0808AB1
:106BA000BDEC21F0809A839AF36A1200D9CFE6FFF8
:106BB000E1CFD9FF010EE126FD0EDBCFE9FFE8288A
:106BC000DBCFEAFFEECF00F0000E00C0DBFFDB50B2
:106BD000E8500BE0DF50E66E1FEC36F0E550FD0E9E
:106BE000DB2AEAE1FE0EDB2AE7D7020EE15EE7CF01
:106BF000D9FF1200D9CFE6FFE1CFD9FF010EE12680
:106C0000FD0EDBCFF6FFE828DBCFF7FF0A00F5CF5C
:106C100000F0000E00C0DBFFDB50E8500BE0DF505F
:106C2000E66E1FEC36F0E550FD0EDB2AE9E1FE0EC4
:106C3000DB2AE6D7020EE15EE7CFD9FF1200D9CFFB
:106C4000E6FFE1CFD9FFB6EC35F0F35001E0FBD71A
:106C5000959A9598F00E95168316FE0EDB50F00B64
:106C6000E83A0F0B83128388839ABDEC21F0808A67
:106C7000BDEC21F0809AF00E8316FE0EDB500F0B58
:106C80008312BDEC21F0808ABDEC21F0809A0F0EBA
:0A6C90009512E552E7CFD9FF12007C
:066C9A004D434850537405
:106CA00061636B2076322E3000426F617264205334
:106CB000657475702E2E2E0020202020202020208C
:106CC000202020202020202000434F4D4D414E44C5
:106CD000532E43474900494E4445582E48544D00D1
:106CE0000D0A0D0A0D4D434850537461636B2044E7
:106CF000656D6F204170706C69636174696F6E209F
:106D000076312E3020284D6963726F636869702078
:106D10005443502F495020537461636B20322E30FE
:106D2000290D0A0D0A09313A204368616E67652012
:106D3000426F6172642073657269616C206E756D5B
:106D40006265722E0D0A09323A204368616E6765EA
:106D50002064656661756C742049502061646472BA
:106D60006573732E0D0A09333A204368616E6765B7
:106D70002064656661756C742067617465776179FC
:106D800020616464726573732E0D0A09343A2043DE
:106D900068616E67652064656661756C74207375E3
:106DA000626E6574206D61736B2E0D0A09353A2091
:106DB000456E61626C65204448435020262049504E
:106DC00020476C65616E696E672E0D0A09363A20A0
:106DD00044697361626C6520444843502026204911
:106DE0005020476C65616E696E672E0D0A09373A4F
:106DF00020446F776E6C6F6164204D50465320695C
:106E00006D6167652E0D0A09383A20536176652059
:106E10002620517569742E0D0A0D0A456E7465722F
:106E20002061206D656E752063686F696365202839
:106E3000312D38293A20000D0A496E76616C69645B
:106E400020696E707574207265636569766564206B
:106E50002D20496E7075742069676E6F7265642E9F
:106E60000D0A507265737320616E79206B6579200D
:106E7000746F20636F6E74696E75652E2E2E0D0A09
:026E8000000010
:0E6E8200FB0EE3CFF6FFFC0EE3CFF7FFFD0E95
:106E9000E3CFF8FFFE0EE3CFE9FFFF0EE3CFEAFFFB
:106EA000F90EE35003E1FA0EE35009E0F90EE306B0
:106EB00002E2FA0EE3060900F550EE5CF1E0F36E33
:106EC0001200D9CFE6FFDACFE6FFFA0EE3CFD9FF03
:106ED000FB0EE3CFDAFFFC0EE3CFE9FFFD0EE3CFBD
:106EE000EAFFE9CFF3FFEACFF4FFF80EE35003E146
:106EF000F90EE35008E0F80EE30602E2F90EE306AD
:106F0000DECFEEFFF2D7FF0EE3CFDAFFE552FF0E42
:106F1000E3CFD9FFE5521200FB0EE3CFF6FFFC0EE4
:106F2000E3CFF7FFFD0EE3CFF8FFFE0EE3CFE9FF5F
:106F3000FF0EE3CFEAFFE9CFF3FFEACFF4FFF90E4C
:106F4000E35003E1FA0EE35009E0F90EE30602E232
:106F5000FA0EE3060900F5CFEEFFF1D71200FE0EA0
:106F6000E3CFE9FFFF0EE3CFEAFFF36AF46AEE52E4
:106F700003E0F34AF42AFBD71200D9CFE6FFDACFB9
:106F8000E6FFFA0EE3CFD9FFFB0EE3CFDAFFFC0EEC
:106F9000E3CFE9FFFD0EE3CFEAFFF80EE35003E194
:106FA000F90EE3500AE0F80EE30602E2F90EE306FA
:106FB000DE50EF5C02E1EE66F0D7F36EFF0EE3CF3A
:106FC000DAFFE552FF0EE3CFD9FFE5521200FE0EC5
:106FD000E3CFE9FFFF0EE3CFEAFFE9CFF3FFEACF0C
:106FE000F4FF610EEF5C05E67B0EEF5C02E7DF0E5F
:086FF000EF16EE52F6E112006B
:086FF800485454502F312E3093
:1070000020353033200D0A0D0A53657276696365A9
:1070100020556E617661696C61626C650D0A000DC8
:107020000A0D0A00485454502F312E30203230308F
:10703000204F4B0D0A436F6E74656E742D7479701A
:10704000653A2000485454502F312E3020343034CB
:10705000204E6F7420666F756E640D0A0D0A4E6FB8
:107060007420666F756E642E0D0A000D0A4E6F77E0
:107070002072756E6E696E67206170706C696361F5
:1070800074696F6E2E2E2E000D0A52656164792090
:10709000746F20646F776E6C6F6164204D5046533F
:1070A00020696D616765202D2055736520586D6FCF
:1070B00064656D2070726F746F636F6C2E0D0A00C3
:1070C0000D0A44484350202620495020476C6561F2
:1070D0006E696E672064697361626C65642E0D0A67
:1070E000000D0A44484350202620495020476C6533
:1070F000616E696E6720656E61626C65642E0D0A53
:10710000000D0A44656661756C74205375626E6586
:1071100074204D61736B2028000D0A44656661750B
:107120006C7420476174657761792041646472658D
:1071300073732028000D0A44656661756C742049DC
:107140005020416464726573732028000D0A5365F2
:0E7150007269616C204E756D626572202800B8
:02715E00545883
:10716000540048544D0047494600434749004A509F
:107170004700434C410057415600746578742F70A6
:107180006C61696E00000000000000000000746582
:1071900078742F68746D6C0000000000000000001F
:1071A0000000696D6167652F676966000000000077
:1071B000000000000000746578742F68746D6C0026
:1071C00000000000000000000000696D6167652F8D
:1071D0006A70656700000000000000000000617038
:1071E000706C69636174696F6E2F6A6176612D7668
:1071F0006D00617564696F2F782D77617665000089
:10720000000000000000485454502F312E3020322E
:107210003030204F4B0D0A436F6E74656E742D74C1
:107220007970653A20000D0A0D0A00474554005058
:0E7230004F535400494E4445582E48544D00CB
:02723E005A0EE6
:10724000F66E000EF76E000EF86E00010900F550A4
:10725000FA6F0900F550FB6F03E1FA6701D03DD0EA
:107260000900F550F56F0900F550F66F0900F5506B
:10727000F76F09000900F550E96E0900F550EA6E54
:10728000090009000900F550F86F0900F550F96F81
:1072900009000900F6CFFCF0F7CFFDF0F8CFFEF0C3
:1072A000F5C0F6FFF6C0F7FFF7C0F8FF0001F8538E
:1072B00002E1F95307E00900F550EE6EF807F8E235
:1072C000F907F9D7FCC0F6FFFDC0F7FFFEC0F8FFD5
:0C72D0000001FA07000EFB5BBFD71200A4
:0472DC000001FF6B43
:1072E0001200D9CFE6FFE1CFD9FF0B0EE126000156
:1072F000FF51000A01E021D0D9CF00F0DACF01F030
:107300000A0E002600C0E6FF01C0E6FFD9CF02F05A
:10731000DACF03F002C0E6FF03C0E6FF3AEC2BF041
:10732000040EE15EF35001E11FD00A0EDB50E86667
:1073300001D01AD00001010EFF6F60EC29F0F3506C
:1073400011E0E66AD9CF00F0DACF01F000C0E6FF25
:1073500001C0E6FF1AEC2CF0E550E550E5500001C5
:10736000FF6B02D0F36A02D0010EF36E0C0EE15EE9
:06737000E7CFD9FF120077
:0A7376005E0ED66EF80ED76E070EFD
:10738000D56ED58EF284F28A1200FEC3F3FFFFC3DE
:10739000F4FF1200F2A40AD0F80ED76E5E0ED66E7D
:0E73A0000301FE4BFF2B0F018978F2941200BF
:0273AE00FF0ED0
:1073B000E350126E480E01D04C0EE76EE72EFED75A
:0E73C000E76AE72EFED7122EF7D70000120064
:0273CE0015EEBA
:1073D00000F025EE00F0F86A118C1FEC39F016EC85
:0673E0001CF0FDD71200B5
:0A73E600FF0EE350E84E1200000015
:0C73F00000D000D000D0E82EFAD7120028
:0473FC0000014C71CF
:0E740000357119710171E170C07088706B7088
:02740E004470C8
:0674100024701F70F86FEC
:02741600000074
:02741800000072
:020000040030CA
:08000000FFFAFCFEFFFEFFFF0A
:00000001FF
